:100000000C9423080C9440080C9440080C9440086D
:100010000C9440080C9440080C9440080C94400840
:100020000C9440080C9440080C9440080C94400830
:100030000C9440080C9440080C9440080C94400820
:100040000C9440080C9440080C94A3140C944008A1
:100050000C94A50A0C9440080C946E0A0C94400869
:100060000C945D1D0C9440080C9440080C944008BE
:100070000C9435100C9440080C9440080D0A000DA7
:100080000A2D2D2D2D2D2D2D2D2D2D2D2D2D2D2DC3
:100090002D2D2D2D2D2D2D2D2D2D2D2D2D2D2D00BD
:1000A0000D0A466F6C6C6F77204D650A0D536F66B5
:1000B00074776172653A5625642E256425632000A5
:1000C0000D0A0D0A48573A20466F6C6C6F772D4D1C
:1000D0006500416E616C6F675F43683020202020AF
:1000E0002020416E616C6F675F43683120202020C3
:1000F0002020416E616C6F675F43683220202020B2
:100100002020416E616C6F675F43683320202020A0
:100110002020416E616C6F675F436834202020208F
:100120002020416E616C6F675F436835202020207E
:100130002020416E616C6F675F436836202020206D
:100140002020416E616C6F675F436837202020205C
:1001500020205542617420202020202020202020B3
:10016000202053797353746174652020202020204F
:100170002020446562756731302020202020202017
:100180002020446562756731312020202020202006
:1001900020204465627567313220202020202020F5
:1001A00020204465627567313320202020202020E4
:1001B00020204465627567313420202020202020D3
:1001C00020204465627567313520202020202020C2
:1001D00020205A656C6C656E7A61686C2020202046
:1001E0002020506F7765724F6E2020202020202025
:1001F000202044656275673138202020202020208F
:10020000202044656275673139202020202020207D
:100210002020446562756732302020202020202075
:100220002020446562756732312020202020202064
:100230002020446562756732322020202020202053
:100240002020446562756732332020202020202042
:100250002020446562756732342020202020202031
:100260002020446562756732352020202020202020
:10027000202044656275673236202020202020200F
:1002800020204465627567323720202020202020FE
:1002900020204465627567323820202020202020ED
:1002A00020204465627567323920202020202020DC
:1002B00020204465627567333020202020202020D4
:1002C00020204465627567333120202020202020C3
:1002D000202021212120494E434F4D504154494275
:1002E0004C4520212121000D0A2055415254302037
:1002F000696E69742E2E2E6F6B006F6B000D0A20D5
:10030000554152543120696E69742E2E2E00546965
:100310006D653A20253032693A253032693A253008
:1003200032692E2530336900446174653A202530E6
:1003300032692F253032692F253034690020202082
:1003400020202020202020202020202020202020AD
:1003500020002020202020202020202020202020BD
:100360002020202020200020204E6F2074696D6501
:100370002064617461212020202020002020202082
:10038000202020202020202020202020202020206D
:1003900000475053205554432054696D65005370F5
:1003A00065656420543A20252B346420636D2F73D7
:1003B00000537065656420453A20252B3464206322
:1003C0006D2F73005370656564204E3A20252B34E1
:1003D0006420636D2F7300536174733A2530326467
:1003E000204669783A3F3F202000536174733A25D4
:1003F000303264204669783A3344202000536174D7
:10040000733A25303264204669783A32442020001D
:10041000536174733A25303264204669783A4E6FDE
:100420006E6500537065656420543A2020202020BA
:100430002020202020202000537065656420453A4C
:100440002020202020202020202020200053706504
:100450006564204E3A2020202020202020202020CB
:1004600020004E6F20475053206461746100416C3E
:10047000743A202563253034642E252E30336420D1
:100480006D004C61743A20256325642E252E33645B
:10049000252E336420646567004C6F6E3A20256317
:1004A00025642E252E3364252E3364206465670071
:1004B000536174733A25303264204669783A3F3F7D
:1004C000202000536174733A2530326420466978E5
:1004D0003A3344202000536174733A25303264204B
:1004E0004669783A3244202000536174733A2530CB
:1004F0003264204669783A4E6F6E6500416C743AFA
:1005000020202020202020202020202020202020EB
:10051000004C61743A202020202020202020202020
:100520002020202020004C6F6E3A20202020202008
:1005300020202020202020202020004E6F20475007
:10054000532064617461002020202020202020207E
:10055000200053573A2025642E2564256300485710
:100560003A20466F6C6C6F772D4D65002B20466FDF
:100570006C6C6F77204D65202B005B25695D005BFF
:1005800025695D006F6B000D0A2055425820696E89
:1005900069742E2E2E006F6B000D0A2041444320FB
:1005A000696E69742E2E2E006F6B000D0A20425565
:1005B00054544F4E20696E69742E2E2E0000002177
:1005C00010422063308440A550C660E7700881293E
:1005D000914AA16BB18CC1ADD1CEE1EFF1311210D6
:1005E0000273325222B5529442F772D6623993188E
:1005F000837BB35AA3BDD39CC3FFF3DEE3622443E2
:100600003420040114E664C774A44485546AA54BDD
:10061000B528850995EEE5CFF5ACC58DD553367275
:100620002611163006D776F6669556B4465BB77A2D
:10063000A719973887DFF7FEE79DD7BCC7C448E501
:10064000588668A7784008611802282338CCC9ED7D
:10065000D98EE9AFF9488969990AA92BB9F55AD415
:100660004AB77A966A711A500A333A122AFDDBDCCD
:10067000CBBFFB9EEB799B588B3BBB1AABA66C8721
:100680007CE44CC55C222C033C600C411CAEED8F1D
:10069000FDECCDCDDD2AAD0BBD688D499D977EB6B5
:1006A0006ED55EF44E133E322E511E700E9FFFBE6D
:1006B000EFDDDFFCCF1BBF3AAF599F788F8891A940
:1006C00081CAB1EBA10CD12DC14EF16FE18010A117
:1006D00000C230E3200450254046706760B983981B
:1006E00093FBA3DAB33DC31CD37FE35EF3B1029067
:1006F00012F322D2323542145277625672EAB5CBE7
:10070000A5A89589856EF54FE52CD50DC5E234C3B6
:1007100024A01481046674476424540544DBA7FABA
:10072000B79987B8975FE77EF71DC73CD7D326F206
:10073000369106B01657667676154634564CD96D06
:10074000C90EF92FE9C899E9898AB9ABA944586556
:100750004806782768C018E1088238A3287DCB5C5A
:10076000DB3FEB1EFBF98BD89BBBAB9ABB754A54A6
:100770005A376A167AF10AD01AB32A923A2EFD0F26
:10078000ED6CDD4DCDAABD8BADE89DC98D267C07F6
:100790006C645C454CA23C832CE01CC10C1FEF3EFA
:1007A000FF5DCF7CDF9BAFBABFD98FF89F176E3646
:1007B0007E554E745E932EB23ED10EF01E4572727F
:1007C0006F7220253032582077726974696E672005
:1007D0006461746120746F207364206361726420AB
:1007E00028523D25303258292E0D0A006F6B000D1E
:1007F0000A20534443206465696E69742E2E2E00CE
:100800004E6F204361726420696E20536C6F742EAA
:10081000000D0A20204361706163697479203D20D6
:100820002569204D42000D0A202053442D4341529A
:10083000442056322E30206F72206C617465720035
:100840000D0A202053442D434152442056312E7826
:10085000006F6B0D0A004572726F722072656164E1
:10086000696E67204353442E004572726F72207286
:10087000656164696E67204349442E0D0A00457224
:10088000726F722073657474696E6720626C6F6337
:100890006B206C656E67746820746F203531322E62
:1008A00000496E6974206572726F722E00496E691C
:1008B000742074696D656F75742E00426164204107
:1008C000636D6434312052313D253032582E00435F
:1008D00061726420697320696E636F6D7061746901
:1008E000626C6520746F20332E33562E004E6F7469
:1008F00020616E2053442D434152442E00426164D6
:1009000020636D64353820523120253032782E0036
:100910004361726420697320696E636F6D706174E6
:1009200069626C6520746F20332E33562E0D0A00D9
:1009300042616420636D64382052372063686563C8
:100940006B207061747465726E2E0D0A00426164D2
:1009500020636D64382052313D253032582E0072AC
:10096000657365742074696D656F7574000D0A2078
:1009700053444320696E69742E2E2E006F6B000D58
:100980000A2053534320696E69742E2E2E002020B6
:100990004D616E756661632E20446174653A202551
:1009A000692F25690D0A0D0A000D0A0025303258FD
:1009B00000202053657269616C204E6F2E3A200032
:1009C000202050726F64756374205265762E3A2031
:1009D00025692E25690D0A00202050726F64756309
:1009E00074204E616D653A2025730D0A0020204168
:1009F00070706C69636174696F6E2049443A202598
:100A0000730D0A000D0A20204D616E7566616374D6
:100A1000757265722049443A2025690D0A004572B5
:100A2000726F7220253032582072656164696E677A
:100A300020646174612066726F6D2073642063614D
:100A40007264202852313D25303258292E0D0A007B
:100A5000202E2E2E6F6B005642523A205061727437
:100A60006974696F6E20697374206E6F74204641DB
:100A700054313620747970652E005642523A204225
:100A80006164206E756D626572206F6620736563A8
:100A9000746F72732E005642523A20536563746F1E
:100AA000722073697A65206E6F7420737570706F31
:100AB000727465642E004572726F72207265616493
:100AC000696E6720746865205642522E0045727226
:100AD0006F722072656164696E6720746865204D6D
:100AE00042522E0053442D4361726420636F756C33
:100AF00064206E6F7420626520696E697469616C30
:100B0000697A65642E000D0A204641543136206909
:100B10006E69742E2E2E005573696E6720646566AB
:100B200061756C742076616C75657321004465662F
:100B300061756C742073657474696E67732066697F
:100B40006C65206372656174656421004552524F83
:100B5000523A204372656174696E6720646566610C
:100B6000756C742073657474696E67732066696C44
:100B70006521006F6B004552524F523A204F70650D
:100B80006E696E672073657474696E677320666939
:100B90006C6521000D0A2053657474696E677320BB
:100BA000696E69742E2E2E000D0A2573203C2D2DA2
:100BB00020756E6B6E6F776E20706172616D6574FB
:100BC00065720D0A000D0A2573203C2D2D20256429
:100BD000206973206F7574206F662072616E67657F
:100BE000205B25642E2E2E25645D000D0A45727251
:100BF0006F7220636C6F73696E67206770782D6603
:100C0000696C650D0A000D0A436C6F73696E67208D
:100C10006770782D66696C650D0A000D0A45727261
:100C20006F72206C6F6767696E6720746F206770E2
:100C3000782D66696C650D0A000D0A4572726F7237
:100C40002067657474696E672066726565206770D9
:100C5000782D66696C65206E616D650D0A000D0A60
:100C60004572726F72206F70656E696E6720677073
:100C7000782D66696C653A2025730D0A000D0A4FC0
:100C800070656E696E67206770782D66696C653A6D
:100C90002025730D0A000D0A4572726F7220636C75
:100CA0006F73696E67206B6D6C2D66696C650D0ADC
:100CB000000D0A436C6F73696E67206B6D6C2D6657
:100CC000696C650D0A000D0A4572726F72206C6FB7
:100CD0006767696E6720746F206B6D6C2D66696C39
:100CE000650D0A000D0A4572726F72206765747493
:100CF000696E672066726565206B6D6C2D66696C28
:100D000065206E616D650D0A000D0A4572726F7285
:100D1000206F70656E696E67206B6D6C2D66696CF7
:100D2000653A2025730D0A000D0A4F70656E696ED5
:100D300067206B6D6C2D66696C653A2025730D0A12
:100D4000003C3F786D6C2076657273696F6E3D2252
:100D5000312E302220656E636F64696E673D2255C7
:100D600054462D38223F3E0D0A3C6B6D6C20786D49
:100D70006C6E733D22687474703A2F2F65617274C3
:100D8000682E676F6F676C652E636F6D2F6B6D6C70
:100D90002F322E32223E0D0A3C446F63756D656E14
:100DA000743E0D0A3C6E616D653E4D696B726F6BF2
:100DB0006F7074657220475053206C6F6767696E5F
:100DC000673C2F6E616D653E0D0A0D0A3C537479C8
:100DD0006C652069643D22464D5F6770732D7374A6
:100DE000796C65223E0D0A3C4C696E655374796CD2
:100DF000653E0D0A3C636F6C6F723E66663030660E
:100E00006630303C2F636F6C6F723E0D0A3C776921
:100E10006474683E323C2F77696474683E0D0A3C06
:100E20002F4C696E655374796C653E0D0A3C2F53E7
:100E300074796C653E0D0A003C2F446F63756D65D7
:100E40006E743E0D0A3C2F6B6D6C3E0D0A003C50DB
:100E50006C6163656D61726B3E0D0A3C6E616D6520
:100E60003E466F6C6C6F774D653C2F6E616D653ED5
:100E70000D0A3C7374796C6555726C3E23464D5F68
:100E80006770732D7374796C653C2F7374796C651E
:100E900055726C3E0D0A003C2F506C6163656D61AC
:100EA000726B3E0D0A003C4C696E65537472696E3C
:100EB000673E0D0A3C74657373656C6C6174653EC6
:100EC000313C2F74657373656C6C6174653E0D0AFB
:100ED0003C616C7469747564654D6F64653E7265E0
:100EE0006C6174697665546F47726F756E643C2FE0
:100EF000616C7469747564654D6F64653E0D0A3C80
:100F0000636F6F7264696E617465733E0D0A000DE4
:100F10000A3C2F636F6F7264696E617465733E0D76
:100F20000A3C2F4C696E65537472696E673E0D0AF8
:100F3000003C3F786D6C2076657273696F6E3D2260
:100F4000312E302220656E636F64696E673D2255D5
:100F500054462D3822207374616E64616C6F6E6527
:100F60003D226E6F22203F3E0D0A3C677078206361
:100F7000726561746F723D22466F6C6C6F774D6560
:100F8000222076657273696F6E3D22312E302220E9
:100F90003E0D0A0D0A3C6D657461646174613E0D1D
:100FA0000A3C6C696E6B20687265663D22687474D9
:100FB000703A2F2F7777772E6D696B726F6B6F702A
:100FC0007465722E6465223E0D0A3C746578743E29
:100FD0004D696B726F4B6F707465723C2F746578DE
:100FE000743E0D0A3C2F6C696E6B3E0D0A3C2F6DF2
:100FF000657461646174613E0D0A0D0A003C2F67DF
:1010000070783E0D0A003C74726B3E0D0A3C6E61B6
:101010006D653E466F6C6C6F774D653C2F6E616DF4
:10102000653E0D0A003C2F74726B3E0D0A003C7445
:10103000726B7365673E0D0A003C2F74726B7365AB
:10104000673E0D0A000011241FBECFEFD0E1DEBFC6
:10105000CDBF13E0A0E0B1E0ECEAFFE802C00590EC
:101060000D92AE39B107D9F71DE0AEE9B3E001C08A
:101070001D92A535B107E1F70E9442080C94D447B0
:101080000C9400002F923F924F925F926F927F924A
:101090008F929F92AF92BF92CF92DF92EF92FF9288
:1010A0000F931F93CF93DF9384B7877F84BF809183
:1010B0006000886180936000109260000E94671950
:1010C00028980E9471140E94820C0E943D1D0E946B
:1010D0005B100E940E1E0E94731E78940E944B3477
:1010E0000E94A6370E94BE3C289A299800D00F92F1
:1010F000ADB7BEB711961C92119780EC90E0139695
:101100009C938E9312970E94391100D000D000D08A
:10111000EDB7FEB73196ADB7BEB711961C9280EA17
:1011200090E0928381831482138281E090E0968321
:10113000858386E690E0908787830E943911EDB71A
:10114000FEB736960FB6F894FEBF0FBEEDBF118204
:101150008FE790E0938382830E943911ADB7BEB7C9
:1011600011961C9211978CE790E013969C938E93A6
:1011700012970E9439110F900F900F900E94161530
:1011800088EE93E00E94ED149093AA038093A90344
:10119000C7EDD5E008ECE02EF12C12E0712EB2E0A4
:1011A000AB2EB12CA1E0CA2ED12C01E0FCE36F2EB6
:1011B000812CE3E09E2E70E7272E77E1372E63E047
:1011C000462E512C0E94DF350E94E33C0E94451EB2
:1011D000882309F0FEC02091A8032093D705198227
:1011E000213009F404C1223009F439C10093A80365
:1011F0008091C001882309F4D8C08091B6069091EF
:10120000B7069093C6058093C5058091B40690916A
:10121000B5069093C8058093C7058091AA06909162
:10122000AB069093CA058093C9058091AC06909156
:10123000AD069093CC058093CB058091B20690913A
:10124000B3069093CE058093CD058091A80690912A
:10125000A9069093D0058093CF058091AE0690911A
:10126000AF069093D2058093D1058091B0069091FE
:10127000B1069093D4058093D3058091B2069091E6
:10128000B3060024969587950794969587950794BD
:10129000982F802D60E771E00E941E44209100018C
:1012A00030910101C901880F991F820F931F680FA8
:1012B000791F769567957695679570930101609390
:1012C00000017093D6056093D505E091A003F091DD
:1012D000A103E436F1057CF4653571050CF0D8C046
:1012E000B0929F03A0929E03CF0101969093A10319
:1012F0008093A003FC0120919E0330919F033093C3
:10130000E6052093E505F093E805E093E7054091B5
:10131000A2035091A303421753070CF06CC0E436AC
:10132000F1050CF468C08091C2039091C303892B2E
:1013300009F061C08091A4039091A503A3E0893EC8
:101340009A070CF45CC084E690E09093C30380930A
:10135000C2034F5F5F4F5093A3034093A20381E00A
:1013600090E09093A5038093A403220F331F22954E
:101370003295307F3227207F3227621773070CF4B3
:1013800045C06A3471050CF441C08091A603909168
:10139000A7038D7F9093A7038093A6031092C001AB
:1013A00080917A00886C80937A000E94E70B0E94FB
:1013B000160E8091A6039091A703892BD1F028984F
:1013C0000E94DF350E94E33C0E94451E882309F4F9
:1013D00002CFF092C303E092C2032091A803213010
:1013E00089F10093A803D092D805C092D705299817
:1013F000FFCE289AE7CE8091A4039091A503A5E0A3
:101400008C3D9A070CF0B1CF0196ABCFE436F105D5
:101410000CF4BBCF90920601809205018091C2032B
:101420009091C303892B21F43092C3032092C2030D
:101430008091A6039091A70382609093A703809365
:10144000A603ACCF8091A6039091A703892B09F046
:10145000C4CE7092A803B092D805A092D70580910F
:10146000A9039091AA030E94F714882309F4C0CE1F
:1014700010919C05113089F08AEF90E00E94ED14E4
:101480009093AA038093A90385B1872585B9B0CE2F
:1014900050929F0340929E0327CF88EE93E00E94D4
:1014A000ED149093AA038093A903EFEFFFEFF0935D
:1014B0009E05E0939D0510939F056092A0051092F4
:1014C000A1051093A2051092A3051092A4051092F5
:1014D000A5051092A6051093B003D6CF1F920F92C8
:1014E0000FB60F9211248F939F93EF93FF938091E8
:1014F00003018823A9F48091BE039091BF03019654
:101500009093BF038093BE03FC01EB5FF94FE08132
:10151000ED3099F08639910581F0E093C60004C062
:101520001092BF031092BE03FF91EF919F918F9194
:101530000F900FBE0F901F9018951092BF0310923E
:10154000BE0381E080930301E8CF1F920F920FB694
:101550000F9211242F933F934F935F936F938F9329
:101560009F93AF93BF93CF93DF93EF93FF936091DC
:10157000C6008091B203882351F43091BB0333231A
:10158000C1F03639C8F01092BB031092B203FF913C
:10159000EF91DF91CF91BF91AF919F918F916F911B
:1015A0005F914F913F912F910F900FBE0F901F9021
:1015B0001895633209F43FC06D3099F0E32FF0E0E5
:1015C000E650FB4F60833F5F3093BB038091BC03C9
:1015D0009091BD03860F911D9093BD038093BC0332
:1015E000D6CFA32FB0E0FD01E850FB4F9081ED0175
:1015F000C750DB4F88814091BC035091BD03491B0C
:101600005109481B51095F705093BD034093BC03BF
:101610002081CA010024880F991F001C880F991F80
:10162000001C892F902D835C281789F01092B2033B
:101630001092BB03ACCF6093FA0481E08093BB03AC
:1016400083E290E09093BD038093BC03A0CF988188
:10165000842F8F73835C981749F7A650BB4F6C9308
:101660003F5F3093B30381E08093B2038091FC0429
:101670008235F1F62CE088E190E00FB6F894A89559
:10168000809360000FBE20936000D2CFCF93DF9392
:10169000BC010097A9F120E030E040E050E0FA0101
:1016A000EB5FF94F8081280F311D4F5F5F4F461769
:1016B0005707A8F33F70C9010024880F991F001C29
:1016C000880F991F001C892F902D835CDB011196D8
:1016D0002F73235CED012196FB01EB5FF94F8083B3
:1016E000AB5FB94F2C93CB5FD94F8DE088831092BD
:1016F0000301809105068093C600DF91CF91089584
:10170000E0E0F0E08DE3A1E0B0E02DE3C2E0D0E066
:10171000E4CF5091B303565009F457C033E043E08F
:101720001EC0972F9D53F0E02295207F892F86952C
:101730008695282BE650FB4F2083E42FEE5F523036
:10174000C1F15350F0E09295990F990F907C6D5331
:10175000962BE650FB4F90834D5F5523A1F1E32F6D
:10176000F0E0E650FB4F80813F5FE32FF0E0E65072
:10177000FB4F20812D533F5FE32FF0E0E650FB4FFE
:1017800070813F5FE32FF0E0E650FB4F60813F5FE9
:10179000922F92959F708D53880F880F892BE42F7D
:1017A000F0E0E650FB4F8083E42FEF5F513009F00B
:1017B000B8CFE3508DEF94E09093B5038093B403DA
:1017C000E093B6030895E42FF4CFE0E0F3CF8091E7
:1017D000B203882309F408950E94890B8091FB04C9
:1017E0008B3611F48091FC048091FC04873609F457
:1017F0005CC08836C0F08C3639F1863709F18836FE
:10180000B1F48FEF80930401E091B403F091B5033C
:10181000808187FD4EC082E08093B1031092BA03AD
:101820001092B90304C0813681F18436D9F0109248
:10183000B5031092B4031092B6031092B203089548
:1018400081E08093AB03F3CF8FEF80930401E091AD
:10185000B403F091B50380818093C50381E0809348
:10186000AD03E5CFE091B403F091B50380812AE0A8
:10187000829FC00111249093B8038093B703892BF2
:10188000B1F281E08093AF03D2CFE091B403F09145
:10189000B503808180930201803218F08FE180933C
:1018A00002018FEF80930401C2CF81E08093AE03E9
:1018B000BECF908190958091C603892B8093C603FB
:1018C00081812AE0829FC00111249093BA03809302
:1018D000B90384E08093B10381E08093AC03A7CF88
:1018E0001F93182F8A3051F08091C00085FFFCCFE4
:1018F0001093C60080E090E01F9108958DE00E9453
:10190000700CF2CF1F931FB7F8948091C1008F77AE
:101910008093C1008091C1008F7B8093C100589A51
:101920005098599A519A1092C5008AE28093C40047
:101930008091C00082608093C00088E18093C100E4
:101940008091C2008F778093C2008091C2008F7B0C
:101950008093C2008091C2008F7D8093C2008091ED
:10196000C2008F7E8093C2008091C200877F8093E7
:10197000C2008091C1008B7F8093C1008091C20022
:1019800084608093C2008091C20082608093C20014
:101990008091C00087FF06C08091C6008091C00082
:1019A00087FDFACF8091C10080688093C10080914B
:1019B000C10080648093C1008091B7039091B80307
:1019C0000E94ED1490939C0680939B061092B203A4
:1019D0001092B5031092B4031092B60381E0809385
:1019E00003011092AE058093AF0585E08093B205A8
:1019F0008AE08093B0051092B1051FBF789400D0A3
:101A00000F92EDB7FEB7118287EE92E09383828347
:101A10000E9439110F900F900F901F910895BF925F
:101A2000CF92DF92EF92FF920F931F93DF93CF93AA
:101A3000CDB7DEB78D852E8593E2909305068F593D
:101A4000809306068C8580930706222379F463E051
:101A500070E0CB010E94460BCF91DF911F910F9157
:101A6000FF90EF90DF90CF90BF900895EF84F888BB
:101A700003E1C02ED12CCC0EDD1E49895A894115B7
:101A8000510529F3022F015063E070E010E062C0BD
:101A9000A12FB0E01F5FFA01AE0DBF1D8C91AF0109
:101AA0004150504009F48BC0E12FF0E01F5FEE0D74
:101AB000FF1DA0814150504009F06DC0002309F482
:101AC0006AC096012E5F3F4FF601E080F18012E080
:101AD000C12ED12CC20ED31EF9014081518101507B
:101AE000382F32953F7090E08F7090702A2F22959A
:101AF000269526952370880F991F880F991F282BEC
:101B0000235CAF73A35C10E08B2D86958695835C78
:101B1000FB01EB5FF94F80838B2D90E08370907019
:101B200082959295907F9827807F9827382B335CF9
:101B3000FB01EA5FF94F3083FB01E95FF94F208336
:101B4000FB01E85FF94FA0836C5F7F4F41155105A2
:101B500009F47FCFF701E10FF11DB0801F5F415005
:101B6000504009F095CF002391F0F6013296D6014E
:101B7000ED90FC9012E0C12ED12CCE0EDF1E019014
:101B8000F081E02D0150309709F04CC010E030E0BA
:101B90002DE3ADE3B9CF382F32953F7090E08F70D1
:101BA00090702A2F2295269526952370880F991FCD
:101BB000880F991F282B235CAF73A35CA5CF00234C
:101BC00071F4382F32953F7090E08F709070880FCD
:101BD000991F880F991F282F235CADE395CFF6013D
:101BE0003296D601ED90FC90A2E0CA2ED12CCE0EFA
:101BF000DF1E4081518101504115510521F0E0E087
:101C0000F0E011E054CF382F32953F7090E08F70A4
:101C10009070880F991F880F991F282F235C10E060
:101C2000ADE372CFA0E0B0E011E036CF0F931F9389
:101C3000DF93CF93CDB7DEB760970FB6F894DEBFD2
:101C40000FBECDBF80910301882309F4B8C08091F5
:101C5000AB03882329F080910301882309F0F0C0A9
:101C60008091B7039091B803892B09F0B3C080919C
:101C7000AC038823A1F180910301882381F1809135
:101C8000B103843008F4A8C10E941F152DB73EB7D8
:101C9000275030400FB6F8943EBF0FBE2DBFEDB7B2
:101CA000FEB7319688E4ADB7BEB711968C938AE043
:101CB000818381E0828388E091E09483838380E55F
:101CC00090E0968385830E940F0DEDB7FEB737969F
:101CD0000FB6F894FEBF0FBEEDBF1092AC0380911B
:101CE000AD03882329F080910301882309F0FCC00B
:101CF000609102016F3F09F441C070E062957295F6
:101D0000707F7627607F76276E527F4F8E010F5F40
:101D10001F4FC80140E150E00E94A0442DB73EB7DC
:101D20002B5030400FB6F8943EBF0FBE2DBFEDB71D
:101D3000FEB7319681E4ADB7BEB711968C938AE0B9
:101D4000818382E0828382E091E09483838381E0D7
:101D500090E0968385831087078380E190E09287E7
:101D600081870E940F0D8FEF80930201EDB7FEB7C0
:101D70003B960FB6F894FEBF0FBEEDBF8091AE0349
:101D8000882329F080910301882309F083C0809182
:101D9000B7039091B803892B09F0E0C08091AF039D
:101DA000882329F080910301882309F0E1C0809104
:101DB000B003882321F0809103018823A9F4609661
:101DC0000FB6F894DEBF0FBECDBFCF91DF911F914C
:101DD0000F91089580919B0690919C060E94F714A4
:101DE000882309F048CF43CF2DB73EB72750304066
:101DF0000FB6F8943EBF0FBE2DBFEDB7FEB73196BC
:101E000083E7ADB7BEB711968C9312E0118381E0E2
:101E1000828380E995E0948383838EE190E09683CA
:101E200085830E940F0D10939C051092B003EDB7AF
:101E3000FEB737960FB6F894FEBF0FBEEDBFBFCF0B
:101E40002DB73EB7275030400FB6F8943EBF0FBEB7
:101E50002DBFEDB7FEB7319686E5ADB7BEB711968B
:101E60008C938AE0818381E082838EEA95E094837B
:101E700083838AE090E0968385830E940F0D109201
:101E8000AB03EDB7FEB737960FB6F894FEBF0FBEA3
:101E9000EDBFE6CE2DB73EB7275030400FB6F894D1
:101EA0003EBF0FBE2DBFEDB7FEB7319687E4ADB78D
:101EB000BEB711968C938AE0818381E0828388EBA0
:101EC00095E0948383838BE090E0968385830E94E2
:101ED0000F0D1092AE03EDB7FEB737960FB6F8941C
:101EE000FEBF0FBEEDBF53CF0E941F152DB73EB7EB
:101EF0002F5030400FB6F8943EBF0FBE2DBFEDB748
:101F0000FEB731968CE4ADB7BEB711968C938AE0DC
:101F1000818383E0828385EC93E09483838321E053
:101F200030E03683258387E091E09087878332878E
:101F3000218788E091E09487838780E590E0968709
:101F400085870E940F0D1092AD03EDB7FEB73F9647
:101F50000FB6F894FEBF0FBEEDBFCACE80919B06B0
:101F600090919C060E94F714882309F01BCF16CF8E
:101F70002DB73EB7275030400FB6F8943EBF0FBE86
:101F80002DBFEDB7FEB7319684E4ADB7BEB711965D
:101F90008C938AE0818381E0828383EC95E0948353
:101FA000838382E490E0968385830E940F0DEDB7D2
:101FB000FEB737960FB6F894FEBF0FBEEDBF809107
:101FC000B7039091B8030E94ED1490939C06809300
:101FD0009B061092AF03EBCE1092C70300D00F9276
:101FE00011E0ADB7BEB711961C93119782ED92E048
:101FF00013969C938E9312970E943911EDB7FEB7FA
:1020000038970FB6F894FEBF0FBEEDBF319688E447
:10201000ADB7BEB711968C93118382E0828381EBBA
:1020200093E09483838381E090E09683858388E0C6
:1020300091E09087878384E190E0928781870E9476
:102040000F0D8091B1038F5F8093B1038150EDB785
:10205000FEB73B960FB6F894FEBF0FBEEDBF8430BF
:1020600008F43BCE1092B10338CE1F920F920FB6F8
:102070000F9211242F933F934F935F936F937F930E
:102080008F939F93AF93BF93EF93FF938091CE0075
:102090000E943D1CFF91EF91BF91AF919F918F9155
:1020A0007F916F915F914F913F912F910F900FBE54
:1020B0000F901F90189500D00F92EDB7FEB71182C8
:1020C0008DEF92E0938382830E9439119FB7F89439
:1020D0008091C9008F778093C9008091C9008F7B60
:1020E0008093C9008091C9008F7D8093C9005A9A5E
:1020F00052985B9A539A1092CD008AE28093CC005A
:102100008091C80082608093C80088E18093C900F4
:102110008091CA008F778093CA008091CA008F7B1C
:102120008093CA008091CA008F7D8093CA008091FD
:10213000CA008F7E8093CA008091CA00877F8093F7
:10214000CA008091C9008B7F8093C9008091CA002A
:1021500084608093CA008091CA0082608093CA0024
:102160008091C8000F900F900F9087FF06C080915C
:10217000CE008091C80087FDFACF8091C9008068A9
:102180008093C9008091C90080648093C9009FBF7B
:10219000789400D00F92EDB7FEB711828AEF92E0EB
:1021A000938382830E9439110F900F900F900895AE
:1021B000982F80919D06813021F0892F0E94700C0C
:1021C00008958091C703E82FF0E0E85FFE4F908309
:1021D0008F5F8093C70381E008951F93182F18160F
:1021E00034F480E30E94D81011501116D4F31F91DB
:1021F00008951F93182F181634F480E20E94D81007
:1022000011501116D4F31F910895EF92FF920F937E
:102210001F93CF93DF937C018B016115710569F0EA
:10222000C0E0D0E0F701EC0FFD1FE4918E2F0E947B
:10223000D8102196C017D107A9F7DF91CF911F9130
:102240000F91FF90EF9008950F931F93CF93DF931B
:102250008C01EB016115710539F0F80181918F0155
:102260000E94D8102197C9F7DF91CF911F910F914C
:1022700008952F923F924F925F926F927F928F922A
:102280009F92AF92BF92CF92DF92EF92FF920F9305
:102290001F93DF93CF93CDB7DEB7EA970FB6F894CD
:1022A000DEBF0FBECDBF61962FAD619762963FAD89
:1022B000629760968FAD609780939D0642E5A42E4D
:1022C000B12CAC0EBD1EC9018C01662477244301DC
:1022D0009E01245D3F4F3AAF29AFF801F490FF20F3
:1022E000A9F0F5E2FF1691F0680103C0F5E2FF16D0
:1022F00039F00894C11CD11CF601F490FF20B1F70D
:10230000B601601B710B09F075C08601FF2009F44E
:1023100095C20F5F1F4F1982EE24552444244A941E
:10232000F8010F5F1F4FF490AE2DB0E0A170B070B8
:1023300025E7F21609F446C08F2D8062883709F42C
:1023400041C06501F0E2FF1609F44DC023E2F21628
:1023500009F495C04AE2F41609F495C05DE2F51659
:1023600009F4A0C0FBE2FF1609F441C02EE2F21608
:1023700009F444C0E0E3FE1609F496C08F2D8153A2
:10238000893008F097C020E030E0C901880F991F1C
:10239000880F991F880F991F220F331F280F391F8D
:1023A0002F0D311D20533040F8010F5F1F4FF49067
:1023B0008F2D80538A3048F3522E560125E7F216AE
:1023C00009F0BACF109709F445C094E0C92ED12C7A
:1023D000CA0CDB1CF5016080718082809380F0E282
:1023E000FF1609F0B3CF8981882309F046C0F9822E
:1023F000560196CFC8010E94051187CFF8010F5FE3
:102400001F4F94919A3209F45FC0892F80538A300C
:1024100080F5692F20E030E0C901880F991F880FEF
:10242000991F880F991F220F331F280F391F260F5E
:10243000311D20533040F8010F5F1F4F6491862FEC
:1024400080538A3048F3A90137FD10C0442EF62E80
:102450005601B4CF82E0C82ED12CCA0CDB1CF5018A
:10246000808191813C01882499246CCF4FEF5FEFEC
:10247000EDCFF92E44245601A1CF560151CF38E0BB
:10248000E32A56014DCFA2E0AA2EB12CAC0CBD1C04
:10249000D6015C9057FE44CF5194B0E1EB2AEFEDAA
:1024A000EE223ECF5601F9CFE4FCE7CFF0E2EF2A6F
:1024B000560136CF28E6F216B9F04CE6F416C1F410
:1024C00051E0E52A56012CCFF2E0AF2EB12CAC0C36
:1024D000BD1CD6014D915C9157FD02C0442E20CF0A
:1024E0004FEF5FEF442E1CCF34E0E32A560118CFA4
:1024F0008F2DF60193E6F91609F405C1843409F429
:1025000072C0843609F471C0893609F46EC08F3404
:1025100009F47AC18F3609F474C1803709F479C19E
:10252000B3E7FB1609F430C155E5F51609F4D4C13B
:1025300085E7F81609F4CCC1E8E5FE1609F4F8C001
:10254000F8E7FF1609F4F4C0FF2009F477C1FC8214
:1025500019822E2D30E03DAB2CAB5601EE2434E039
:10256000232E312C2C0E3D1E81E091E0E0E021E095
:10257000C22ED12C2981222381F18F5F482E4E0E4D
:102580008CA99DA98073907098AF8FAB892B29F48B
:10259000852D84190E94F91029812223B9F49CA960
:1025A00096FD8CC1EFA9F8ADB09709F482C18E2DCC
:1025B0000E94ED10C101B6010E942411FCA9F4FF94
:1025C0008CCE852D84190E94F91087CECE010196FC
:1025D00061E070E00E942411E5CF5CA956FFCECFE8
:1025E000892F8E5FCBCFB1E0EB2AE0FE54C1B4E07F
:1025F000AB2EB12CAC0CBD1CF601608071808280CA
:10260000938097FC3BC1BAE0BEAB47FC02C05FEDD4
:10261000E5227CE2272E312C2C0E3D1E6114710424
:102620008104910409F452C09EA9892F90E0A0E092
:10263000B0E088AB99ABAAABBBAB6CE2C62ED12C99
:10264000CC0EDD1E6CA67DA68EA69FA62AC050E3EA
:10265000352E360ED6013E926D016CA57DA58EA558
:102660009FA528A939A94AA95BA90E944544B90197
:10267000FA01C901DA013C014D012CA53DA54EA589
:102680005FA588A999A9AAA9BBA9281739074A074C
:102690005B0708F440C0CB01DF018CA79DA7AEA764
:1026A000BFA76CA57DA58EA59FA528A939A94AA974
:1026B0005BA90E9445446A3050F247E5342E360E3D
:1026C00048E5F41639F65FED3522C4CF442089F48D
:1026D000AE2DB0E0BDABACAB80E090E0442DE42E7D
:1026E000E91AE7FCC4C0EE2DC82EDD24C7FCD09447
:1026F00041CF3EA9232F30E040E050E028AB39AB7A
:102700004AAB5BAB9ACFA2E0B0E0CA0EDB1E808181
:102710008C8319821ECF9EA99830D1F0AE2DB0E0E7
:10272000BDABACABB9ADBC198B2F9B2F1601D6CF6F
:10273000E3FE1AC06114710481049104A9F020E43D
:10274000E22A8F2D30E13EAB1982F82E56015DCF83
:10275000EE2DF0E0FDABECABE3FC0AC0F9ADFC19EB
:102760008F2F9F2F1601BACF8F2D40E14EABECCFAC
:1027700020E3321609F45CC0F60140E3429389ADD0
:102780008E1B982F1F01AACFF601208031802114C3
:10279000310489F4F8E2FC832EE62D8335E73E838D
:1027A0008CE68F83888789E289871A86F4E02F2E4A
:1027B000312C2C0E3D1E47FC1CC0442D552747FDD7
:1027C0005095C10160E070E00E94A944009719F0A3
:1027D000821948160CF4842DE2E0AE2EB12CAC0C1C
:1027E000BD1C1982982F4E2D50E05DAB4CAB40E0E4
:1027F00076CFF10101900020E9F731978E2F8219F1
:10280000EBCF28E02EABA0CF31E0E32A48E04EAB7F
:102810009BCF82E090E0C80ED91E808191813C015F
:102820008824992490E4E92A88E7A0E1AEAB8CCF14
:1028300039AD3C19832F932F160150CFEA960FB66E
:10284000F894DEBF0FBECDBFCF91DF911F910F91E6
:10285000FF90EF90DF90CF90BF90AF909F908F90C0
:102860007F906F905F904F903F902F900895C82E6B
:10287000DD24C7FCD094EE24E0E07CCE90948094DC
:1028800070946094611C711C811C911CEDE2E983C1
:10289000FAE0FEABBACEA2E0AA2EB12CAC0CBD1C65
:1028A000D6018D919C913C01882477FC8094982CD2
:1028B000A8CE852D84190E94ED1079CEA0E3AA83BD
:1028C000FB82CE01029662E070E00E9424116ACE83
:1028D0008F2D9AE09EAB38CFA1E0EA2ABAE0BEABDA
:1028E00033CF9FB7F8943F9A479884B58C7084BDD6
:1028F00085B5877385BD85B5887F826085BD16BC2B
:10290000EEE6F0E08081897F808380818160808332
:1029100010929F0610929E061092A0061092A10699
:102920001092A2061092A3061092A4061092A60678
:102930001092A5061092A7061092C1031092C00330
:102940009FBF789408951F920F920FB60F92112493
:102950002F933F938F939F938091C40381508093D3
:10296000C4038F5F61F489E08093C4038091C00346
:102970009091C10301969093C1038093C00380910D
:10298000C2039091C303892BF9F08091C203909107
:10299000C30301979093C3038093C2032091C203A2
:1029A0003091C30380910501909106018223932306
:1029B000892B89F447989F918F913F912F910F9088
:1029C0000FBE0F901F9018958FEF9FEF9093060109
:1029D00080930501EFCF479AEECF2091C00330914D
:1029E000C10321503040280F391FC901089520919B
:1029F000C0033091C103821B930B80709078892FA4
:102A000008952091C0033091C10321503040280F18
:102A1000391F8091C0039091C103A901481B590B34
:102A2000CA01807090789923A1F30895E8E0F1E05D
:102A300080E2819391E0E835F907D9F708958F9204
:102A40009F92AF92BF92CF92DF92EF92FF920F933D
:102A50001F93CF93DF938091C60390E080FF08C05F
:102A60002091C503222309F4C5C021502093C5033A
:102A70003091070181FF08C02091C503231709F495
:102A8000C5C22F5F2093C50383709070039711F424
:102A90001092C503E8E0F1E080E2819391E0E8352F
:102AA000F907D9F72091C503321718F43093C503FD
:102AB000232F2A3008F082C081E18093C70300D021
:102AC00000D00F92EDB7FEB7319681E0ADB7BEB73B
:102AD00011968C938FE795E09283818323831482F0
:102AE0000E9439110F900F900F900F900F9010913E
:102AF000C503113009F4CBC0113008F070C010923A
:102B0000C70300D00F9211E0EDB7FEB711838CE63A
:102B100095E0938382830E94391184E18093C703F7
:102B2000ADB7BEB711961C9311978EE595E013963D
:102B30009C938E9312970E94391188E28093C70369
:102B400000D000D000D0EDB7FEB73196ADB7BEB71C
:102B500011961C9382E595E09283818314821382FF
:102B600081E090E09683858386E690E09087878376
:102B70000E9439118CE38093C703EDB7FEB73696F8
:102B80000FB6F894FEBF0FBEEDBF118387E495E04A
:102B9000938382830E9439110F900F900F901092AF
:102BA000C603DF91CF911F910F91FF90EF90DF90BF
:102BB000CF90BF90AF909F908F90089580E18093C9
:102BC000C70300D000D00F92EDB7FEB7319681E079
:102BD000ADB7BEB711968C938AE795E07DCF1230E2
:102BE00009F4A4C1133059F0115010930701109249
:102BF000C503D5CF309107013093C5033BCF109269
:102C0000C70300D00F9211E0EDB7FEB7118381E941
:102C100093E0938382830E9439110F900F900F905D
:102C20008091A706882309F0F4C184E18093C7034B
:102C300000D00F92ADB7BEB711961C9311978CE7D9
:102C400093E013969C938E9312970E94391188E219
:102C50008093C703EDB7FEB7118387E693E09383B4
:102C600082830E9439118CE38093C703ADB7BEB74E
:102C700011961C93119782E593E013969C938E9383
:102C800012970E9439110F900F900F9088CF80916A
:102C90006D04882309F456C280915004823009F4EF
:102CA000CFC2833009F4BDC2882309F488C21092D0
:102CB000C70300D000D00F92EDB7FEB73196ADB785
:102CC000BEB711961C9380EB94E092838183809130
:102CD0004F04838314820E9439110F900F900F903C
:102CE0000F900F90E0904104F09042040091430453
:102CF0001091440417FD82C23BE2C32ED12CC801BF
:102D0000B70120E836E948E950E00E946744B62E52
:102D1000A72E982E892E84E18093C703EDB7FEB7C6
:102D20003B970FB6F894FEBF0FBEEDBFCDB7DEB731
:102D3000219681E0ADB7BEB711968C9389E994E0F6
:102D40009A838983DC82CB82C801B70120E836E907
:102D500048E950E00E946744C90137FD5EC29E8386
:102D60008D836B2D7A2D892D982D20E137E240E05F
:102D700050E00E946744C90137FD7DC298878F8368
:102D80006B2D7A2D892D982D20E137E240E050E01F
:102D90000E9467442AE030E040E050E00E9467442F
:102DA000C90137FD64C29A8789870E943911E09072
:102DB0004504F09046040091470410914804EDB793
:102DC000FEB73B960FB6F894FEBF0FBEEDBF17FDE2
:102DD0001CC29BE2C92ED12CC801B70120E836E9FC
:102DE00048E950E00E946744B62EA72E982E892EFF
:102DF00088E28093C7038DB79EB70B970FB6F89400
:102E00009EBF0FBE8DBFCDB7DEB7219681E0ADB7B7
:102E1000BEB711968C9382E894E09A838983DC8212
:102E2000CB82C801B70120E836E948E950E00E94AA
:102E30006744C90137FD17C29E838D836B2D7A2DA0
:102E4000892D982D20E137E240E050E00E94674450
:102E5000C90137FD38C298878F836B2D7A2D892D54
:102E6000982D20E137E240E050E00E9467442AE0DC
:102E700030E040E050E00E946744C90137FD1FC2C6
:102E80009A8789870E943911E0904904F0904A049A
:102E900000914B0410914C04EDB7FEB73B960FB672
:102EA000F894FEBF0FBEEDBF17FDACC12BE230E0C2
:102EB0008CE38093C7038DB79EB709970FB6F8943C
:102EC0009EBF0FBE8DBFCDB7DEB7219681E0ADB7F7
:102ED000BEB711968C938EE694E09A8389833C83E7
:102EE0002B83C801B70128EE33E040E050E00E9498
:102EF0006744C90137FDB3C19E838D83C801B70103
:102F000028EE33E040E050E00E946744CB0177FDBB
:102F100080C198878F830E943911EDB7FEB739962B
:102F20000FB6F894FEBF0FBEEDBF39CE80916D0491
:102F3000882309F4C9C080915004823009F4AFC1DC
:102F4000833009F49CC1882309F448C11092C70357
:102F500000D000D00F92EDB7FEB7319681E0ADB74B
:102F6000BEB711968C9387ED93E092838183809115
:102F70004F04838314820E94391184E18093C70334
:102F8000EDB7FEB7319611E0ADB7BEB711961C9301
:102F900084EC93E092838183809155049091560450
:102FA000948383830E94391188E28093C703EDB72D
:102FB000FEB73196ADB7BEB711961C9381EB93E087
:102FC000928381838091590490915A0494838383DE
:102FD0000E9439118CE38093C703EDB7FEB7319699
:102FE000ADB7BEB711961C938EE993E092838183AF
:102FF00080915D0490915E04948383830E943911D3
:103000000F900F900F900F900F90C9CD1092C503A5
:103010003BCD84E18093C70300D00F92EDB7FEB79C
:1030200011838DE393E0938382830E94391188E2B8
:103030008093C70300D000D000D0EDB7FEB7319623
:10304000ADB7BEB711961C9388E293E0928381835B
:103050008091A006838314828091A10685831682C5
:1030600080919E0690919F06908787830E943911D8
:103070008CE38093C70300D0EDB7FEB73196ADB7B0
:10308000BEB711961C938EE093E09283818380916A
:10309000A206838314828091A30685831682809181
:1030A000A406878310868091A5069091A606928734
:1030B00081870E943911EDB7FEB73B960FB6F894A1
:1030C000FEBF0FBEEDBF6BCD1092C70300D00F92B5
:1030D00011E0ADB7BEB711961C93119782E694E04C
:1030E00013969C938E9312970E94391184E18093DA
:1030F000C703EDB7FEB711838DE494E09383828319
:103100000E94391188E28093C703ADB7BEB711960C
:103110001C93119788E394E013969C938E931297D7
:103120000E9439118CE38093C703EDB7FEB711837A
:1031300083E294E0938382830E9439110F900F9071
:103140000F902DCD1092C70300D00F92ADB7BEB730
:1031500011961C9311978BE395E013969C938E9395
:1031600012970E94391184E18093C703EDB7FEB72F
:10317000118386E295E0938382830E94391188E26D
:103180008093C703ADB7BEB711961C93119781E129
:1031900095E013969C938E9312970E9439118CE3BD
:1031A0008093C703EDB7FEB711838CEF94E0938350
:1031B00082830E9439110F900F900F90F0CC1092E3
:1031C000C70300D000D00F92EDB7FEB73196ADB770
:1031D000BEB711961C9389EE94E077CD1092C70389
:1031E00000D000D00F92EDB7FEB7319681E0ADB7B9
:1031F000BEB711968C9380E194E0B7CE2DE2C22E3B
:10320000D12C7DCD2DE230E053CE8DE2C82ED12CD5
:10321000E3CD909581959F4F7CCE909581959F4F62
:103220009ECD1092C70300D000D00F92EDB7FEB72D
:103230003196ADB7BEB711961C9383EC94E045CDA3
:103240001092C70300D000D00F92EDB7FEB73196B1
:10325000ADB7BEB711961C9386ED94E036CD909530
:1032600081959F4F49CE909581959F4FE5CD909543
:1032700081959F4F98CD909581959F4F7FCD1092CE
:10328000C70300D000D00F92EDB7FEB7319681E0B2
:10329000ADB7BEB711968C938AEE93E066CE1092CE
:1032A000C70300D000D00F92EDB7FEB7319681E092
:1032B000ADB7BEB711968C938DEF93E056CE909537
:1032C00081959F4FDDCD909581959F4FC4CD209ADC
:1032D000299A219A289A08959C0160E971E00E9438
:1032E0001E44892B81F0C90183709070892B19F0DD
:1032F00040E0842F089540E0C90164E670E00E9438
:103300001E44892B09F041E0842F08952F923F92AB
:103310004F925F926F927F928F929F92AF92BF92E5
:10332000CF92DF92EF92FF920F931F93DF93CF9391
:10333000CDB7DEB72E970FB6F894DEBF0FBECDBF68
:103340009E878D878091FC03882321F08091D30391
:1033500082FD1DC0AD85BE8519961C922E960FB6B6
:10336000F894DEBF0FBECDBFCF91DF911F910F91BB
:10337000FF90EF90DF90CF90BF90AF909F908F9095
:103380007F906F905F904F903F902F900895809125
:10339000D30383FFDFCF6091C8037091C90380918D
:1033A000CA039091CB0328EE33E040E050E00E9446
:1033B000454479018A018091D0039091D1039C0109
:1033C000442737FD4095542F6FE0E616F1040105C0
:1033D000110508F04AC12150304040405040D8010A
:1033E000C7018F58954CA64FBF4F89839A83AB83F3
:1033F000BC8349015A01880C991CAA1CBB1C880C6F
:10340000991CAA1CBB1C880C991CAA1CBB1C821AE8
:10341000930AA40AB50A69817A818B819C8120E88C
:1034200031E541E050E00E944544820E931EA41E07
:10343000B51E83E897E0ABE0B0E0880E991EAA1EA7
:10344000BB1EC501B40121EB3AE342E050E00E940B
:1034500045446D837E838F8398872CEA3EE840E065
:1034600050E00E94454469877A878B879C8725EBCB
:1034700035E040E050E00E9445446B017C0197E458
:10348000C91694E0D90690E0E90690E0F90608F440
:10349000D5C023E0622E712C97E4292E94E0392EBA
:1034A000412C512CC501B40121EB3AE342E050E03C
:1034B0000E94454480E991E0289F8001299F100DDA
:1034C000389F100D11240F5F1F4F6D817E818F81FA
:1034D00098852CEA3EE840E050E00E94454484E6AE
:1034E00090E0FC012E9FC0012F9F900D3E9F900DFC
:1034F0001124080F191F69857A858B859C8525EB1A
:1035000035E040E050E00E944544220F331F220F77
:10351000331F020F131F060D171DAD85BE850D93BA
:103520001C930894C11CD11CE11CF11CC218D308C7
:10353000E408F508C8010E946C19882309F47BC0CF
:1035400088E591E0FC0120E080819181A281B38136
:103550008C159D05AE05BF0508F067C08481958177
:10356000A681B7818C159D05AE05BF0508F45DC029
:103570002F5FAD85BE8512962C938081BC2DB81B24
:10358000ED85FE85B38369817A818B819C8120E8FA
:1035900031E541E050E00E944544162F072FF82EF8
:1035A000E92E20E13EE040E050E00E944544AD8538
:1035B000BE8514962C93612F702F8F2D9E2D20E1A8
:1035C0003EE040E050E00E944544162F072FF82EC1
:1035D000E92E2CE330E040E050E00E944544ED85C8
:1035E000FE852583612F702F8F2D9E2D2CE330E0DB
:1035F00040E050E00E944544AD85BE8516966C9330
:103600006091C8037091C9038091CA039091CB0364
:1036100028EE33E040E050E00E944544ED85FE8511
:103620007087678381E0818799CE2F5F34962C3035
:1036300009F08ACFA8CF8CE891E084CFC701B6010A
:103640002DE631E040E050E00E94454439018DE62E
:1036500091E0DC012A9FC0012B9F900D3A9F900DB5
:1036600011241C01442455241DCFC801B7016F50FB
:1036700070408040904069837A838B839C83B9CE6D
:103680001F9380917A0490917B040E94F714882301
:10369000D9F01092790484E690E00E94ED149093A2
:1036A0007B0480937A0480917904823058F0809171
:1036B000FC03813079F082E08093FC03809319044D
:1036C00080933E041F910895809179048F5F8093C9
:1036D0007904E1CF80911904813069F710913E049B
:1036E000113049F780913F049091400401969093E6
:1036F000400480933F0480916D048130E1F2109288
:103700006D048091D30380934E048091F7038093DE
:103710004F048091D203809350048091E0039091F4
:10372000E103A091E203B091E303809351049093ED
:103730005204A0935304B09354048091F0039091E9
:10374000F103A091F203B091F30380936904909385
:103750006A04A0936B04B0936C048EE996E00E9417
:1037600086198091010490910204A0910304B09104
:1037700004048093410490934204A0934304B093C3
:1037800044048091050490910604A0910704B0912F
:1037900008048093450490934604A0934704B09393
:1037A000480480910D0490910E04A0910F04B091F3
:1037B00010048093490490934A04A0934B04B0935F
:1037C0004C0410934D048091220490912304A09105
:1037D0002404B09125048093590490935A04A09333
:1037E0005B04B0935C0480911E0490911F04A0912F
:1037F0002004B09121048093550490935604A09323
:103800005704B09358048091260490912704A09106
:103810002804B0912904B095A095909581959F4F6B
:10382000AF4FBF4F80935D0490935E04A0935F04FD
:10383000B093600480912E0490912F04A0913004E5
:10384000B09131048093610490936204A093630467
:10385000B09364048091320490913304A0913404B5
:10386000B09135048093650490936604A093670437
:10387000B093680410936D041ECF482F8091780494
:10388000843009F4B4C0853070F0863009F476C015
:103890008630E0F1873009F469C0883009F459C0F6
:1038A000109278040895813009F49AC0813030F480
:1038B000453B09F4AEC0109278040895823009F4B3
:1038C00088C0833069F7463009F4B8C0423109F442
:1038D000A4C0423081F78DEF93E0909373048093FE
:1038E00072044D96909371048093700401979093A5
:1038F0006F0480936E0484E080937804842F8F5F3C
:10390000809375048F5F809374040895342F20E0B2
:103910008091760490917704820F931F909377049F
:103920008093760490917504940F90937504809120
:103930007404890F80937404E0916E04F0916F0415
:103940008081813009F494C0108286E080937804ED
:10395000089580917404481709F481C0E0916E04C1
:10396000F0916F041082109278040895809175048C
:103970004817A1F788E0809378040895E0917204D5
:10398000F09173048091700490917104E817F90725
:1039900008F091CF4193F0937304E09372049091F7
:1039A0007504940F9093750480917404890F80932B
:1039B0007404809176049091770401979093770432
:1039C00080937604892B09F06DCF87E0809378048B
:1039D0000895413009F06FCF83E080937804089513
:1039E000423609F068CF82E08093780408954093CE
:1039F00076041092770480917504840F8093750487
:103A000090917404980F9093740485E080937804E7
:103A1000089581E08093780408958AE194E090937A
:103A2000730480937204859690937104809370045C
:103A3000019790936F0480936E045DCF88EC93E0C0
:103A40009093730480937204C5969093710480934D
:103A50007004019790936F0480936E044CCFE091B3
:103A60006E04F0916F0481E080830E94401B23CF9D
:103A7000109278040E94401B089500D00F92EDB779
:103A8000FEB7118287E895E0938382830E94391103
:103A90001092FC031092190410923E0410926D04CF
:103AA000EDB7FEB7118284E895E0938382830E948C
:103AB00039110F900F900F9008951F920F920FB62B
:103AC0000F9211242F938F939F9380917C04282F22
:103AD0002F5F20937C04833009F494C08430F8F085
:103AE000853009F45BC0853058F1863009F472C026
:103AF000873009F45FC010927D0410927C0481E04D
:103B00008093C00180917C00807E80937C009F9197
:103B10008F912F910F900FBE0F901F9018958130AD
:103B200009F464C0823070F180917800909179003E
:103B30009093AB068093AA0683E080937D040BC02C
:103B400080917800909179009093B3068093B206AB
:103B500085E080937D0480917C00807E90917D043F
:103B6000892B80937C00222391F280917A00886CCB
:103B700080937A009F918F912F910F900FBE0F909D
:103B80001F90189580917800909179009093B706D6
:103B90008093B60681E080937D04DDCF809178002C
:103BA000909179009093A9068093A80686E080936F
:103BB0007D04D1CF80917800909179009093B106E7
:103BC0008093B00610927D0410927C0481E0809373
:103BD000C00198CF80917800909179009093AF06C2
:103BE0008093AE0687E080937D04B5CF8091780006
:103BF000909179009093B5068093B40682E080930B
:103C00007D04A9CF80917800909179009093AD06C2
:103C10008093AC0684E080937D049DCF1F931FB7F3
:103C200000D00F92EDB7FEB7118289E995E093833A
:103C300082830E943911F89411B812B88FEF8093E3
:103C40007E00ECE7F0E080818F7180838081807E50
:103C50008083AAE7B0E087E08C93EBE7F0E0808117
:103C6000887F80838C91886C8C931FBF7894EDB78C
:103C7000FEB7118286E995E0938382830E94391111
:103C80000F900F900F901F9108951F9380917E04C5
:103C900090917F040E94F7148823D1F036990AC0CE
:103CA00080918004982F9F5F909380048823A1F4D3
:103CB00011E003C01092800410E082E390E00E94C3
:103CC000ED1490937F0480937E04812F1F910895BB
:103CD00010E0812F1F9108959A3071F787E080934B
:103CE000800411E0EACF00D00F92EDB7FEB7118249
:103CF0008BEA95E0938382830E943911469A3E981D
:103D00000F900F900F9082E390E00E94ED1490933B
:103D10007F0480937E0400D00F92EDB7FEB711822E
:103D200088EA95E0938382830E9439110F900F9067
:103D30000F900895EF92FF920F931F93CF93DF930D
:103D4000EC017A018B01411551056105710559F1AD
:103D500040E050E060E070E0E0E0F0E03E2F22273D
:103D6000EF2FFF27DE01A40FB51F8C9190E0E8270D
:103D7000F927EE0FFF1FE354FA4F0190F081E02D79
:103D8000E227F3274F5F5F4F6F4F7F4F4E155F0561
:103D90006007710718F3CF01DF91CF911F910F9149
:103DA000FF90EF900895E0E0F0E0F5CF84B1806BF4
:103DB00084B926982C9A82E58CBD8DB581608DBD25
:103DC0002A9A229808952C9A1CBC1DBC08958FEF46
:103DD0008EBD0DB407FEFDCF8EB508958EBD0DB41A
:103DE00007FEFDCF08952C9A08952C9808951F93EF
:103DF000CF93DF93EC01411551056105710519F170
:103E000030E020E019E0FE01E30FF11DE08190E0D9
:103E100001C0EE0F220F822F8E2787FD21279F5F83
:103E20009830B9F73F5F832F90E0A0E0B0E08417AF
:103E30009507A607B70738F3822F880F8160DF91B7
:103E4000CF911F91089581E0FACF00D00F92EDB786
:103E5000FEB711828FEE97E0938382830E9439111F
:103E60000F900F900F900E94E31E1092B8061092D0
:103E7000BA061092BB061092BC061092BD061092B4
:103E8000B90600D00F92EDB7FEB711828CEE97E025
:103E9000938382830E9439110F900F900F9080E0DE
:103EA0000895CF92DF92EF92FF920F931F93DF93CB
:103EB000CF9300D000D000D0CDB7DEB76C0100D0DA
:103EC00000D00F92EDB7FEB73196ADB7BEB71196E1
:103ED0001C9284E09AE092838183D6018C91838343
:103EE00014820E943911F601818192819A8389831B
:103EF0001B820DB71EB70F5F1F4FADB7BEB7119630
:103F00001C928DEE99E0F801928381837E010894E2
:103F1000E11CF11CF482E3820E943911D701F60101
:103F2000339685E001900D928150E1F71E82D80111
:103F30001C9288ED99E012969C938E93119714969B
:103F4000FC92EE9213970E943911F601208500D061
:103F5000EDB7FEB73196ADB7BEB711961C9280ECA7
:103F600099E092838183822F82958F70838314825C
:103F700030E02F703070368325830E9439110F9006
:103F80000F900F900F90EDB7FEB7118281EB99E083
:103F9000938382830E94391100D0EDB7FEB731962A
:103FA000ADB7BEB711961C920CEA19E012830183DB
:103FB000D60119968C91838314820E943911EDB732
:103FC000FEB73196ADB7BEB711961C92128301832E
:103FD000D6011A968C91838314820E943911EDB711
:103FE000FEB73196ADB7BEB711961C92128301830E
:103FF000D6011B968C91838314820E943911EDB7F0
:10400000FEB73196ADB7BEB711961C9212830183ED
:10401000D6011C968C91838314820E9439110F90D3
:104020000F90EDB7FEB7118289EA99E093838283FE
:104030000E943911D6011E962C9100D000D0EDB708
:10404000FEB73196ADB7BEB711961C928EE899E0D7
:1040500092838183822F90E08F709070948383830A
:10406000D6011D968C9190E082959295907F98272D
:10407000807F982722952F7030E0822B932B8053DE
:10408000984F968385830E943911EDB7FEB7379616
:104090000FB6F894FEBF0FBEEDBF26960FB6F8948C
:1040A000DEBF0FBECDBFCF91DF911F910F91FF906B
:1040B000EF90DF90CF9008950F931F93CF93DF93EE
:1040C0008C010E94F51EC8010E94ED14EC010E94B3
:1040D000E71E082FCE010E94F714882311F40F3F2A
:1040E000B1F7802FDF91CF911F910F910895CF925B
:1040F000DF92EF92FF920F931F93DF93CF9300D045
:1041000000D000D0CDB7DEB780648983872F992790
:10411000AA27BB278A836B835C834D838E010F5F45
:104120001F4FC80145E050E060E070E00E94F71EBC
:104130008E830E94F31E8FEF0E94EE1E0E94F51EDA
:1041400084EF91E00E945C2057E0C52ED12CCC0E6C
:10415000DD1E4AE0E42EF12CF80181918F010E94CE
:10416000EE1EC7010197F1F70C151D05A9F70E9476
:10417000E71E8F3F61F401E010E00E94E71E0F5F31
:104180001F4FF1E0063F1F0711F08F3FB1F3269656
:104190000FB6F894DEBF0FBECDBFCF91DF911F9158
:1041A0000F91FF90EF90DF90CF900895EF92FF92E4
:1041B0000F931F93CF93DF938B019C017A01F9E05A
:1041C000000F111F221F331FFA95D1F788E1B901A3
:1041D000A8010E947720882309F071C0C0E0D0E0D8
:1041E0000E94E71E2196C431D105D1F7C70140E0F6
:1041F00052E060E070E00E949A1E182F092F8EEFA7
:104200000E94EE1EC0E0D0E0F701EC0FFD1F8081A0
:104210000E94EE1E219682E0C030D807A9F7802FB9
:104220000E94EE1E812F0E94EE1E0E94E71EC1E03A
:10423000D0E008C00E94E71E91E0C53FD90709F40D
:104240004EC02196282F30E0C901817190700197EE
:1042500089F7C9018F7190708B309105B1F18D3163
:10426000910509F446C00597A1F10CE04CE050E03F
:10427000ADB7BEB717970FB6F894BEBF0FBEADBFB0
:10428000EDB7FEB7319611961C928DEB97E09283B5
:10429000818354834383368325830E9439118DB7EC
:1042A0009EB707960FB6F8949EBF0FBE8DBF802FA6
:1042B000DF91CF911F910F91FF90EF900895282FDC
:1042C00030E004E044E050E0D3CF08E048E050E0C4
:1042D000CFCF80ED97E00E945C208F3F71F0282FB8
:1042E00030E007E047E050E0C3CF0E94E71E212FF7
:1042F00030E009E049E050E0BBCF8DE040E050E025
:1043000060E070E00E947720182F882341F00E941F
:10431000E71E212F30E004E044E050E0A9CF0E94E6
:10432000E71E182F882309F700E0C1CFCF92DF9254
:10433000EF92FF920F931F93CF93DF9369010E9437
:104340007720882369F50E94E71E282F807F09F4D3
:104350004DC02E3FC1F7E114F1040105110589F0AC
:10436000C0E0D0E00E94E71EF601EC0FFD1F808345
:104370002196CE01A0E0B0E08E159F05A007B10701
:1043800088F30E94E71E0E94E71E10E0812FDF9154
:10439000CF911F910F91FF90EF90DF90CF900895F4
:1043A000282F14E044E050E08DB79EB707970FB672
:1043B000F8949EBF0FBE8DBFEDB7FEB73196ADB777
:1043C000BEB711961C928EE19AE09283818354834A
:1043D0004383258316820E9439118DB79EB70796B5
:1043E0000FB6F8949EBF0FBE8DBFD0CF1AE04AE043
:1043F00050E0DACFEF92FF920F931F937B018C0175
:104400009A01B9E0EE0CFF1C001F111FBA95D1F7FD
:1044100081E1B801A701E12CA2E0FA2E012D112DB6
:104420000E9496211F910F91FF90EF900895EF92B7
:10443000FF920F931F939C0189E040E050E060E001
:1044400070E090E1E92EF12C012D112D0E949621B2
:104450001F910F91FF90EF900895EF92FF920F93AD
:104460001F939C018AE040E050E060E070E0E0E1F2
:10447000EE2EF12C012D112D0E9496211F910F91EE
:10448000FF90EF900895DF92EF92FF920F931F93AA
:10449000D82E7A018B0187E340E050E060E070E0C5
:1044A0000E94772087FD05C08D2DB801A7010E94CD
:1044B00077201F910F91FF90EF90DF900895CF929A
:1044C000DF92EF92FF920F931F93DF93CF9300D071
:1044D00000D000D0CDB7DEB71A999CC000D00F92A3
:1044E000ADB7BEB711961C9211978FE799E013965E
:1044F0009C938E9312970E9439110F900F900F90FA
:104500000E94D61E00D00F92EDB7FEB711828CE745
:1045100099E0938382830E943911ADB7BEB711969B
:104520001C9211978DE699E013969C938E931297A7
:104530000E9439111092B8060F900F900F900E94B0
:10454000F31E00E010E08FEF0E94EE1E0F5F1F4F82
:104550000F301105C1F780E040E050E060E070E00E
:104560000E9477208983813099F001E010E080E09B
:1045700040E050E060E070E00E9477200F5F1F4F46
:10458000B1E0063F1B0709F410C1813081F7898330
:1045900088E04AEA51E060E070E00E947720282F2E
:1045A00087FDA0C0898382FF5CC081E08093B9064B
:1045B0008AE340E050E060E070E00E947720282F1E
:1045C00087FDE6C082FDA7C089838E010E5F1F4F65
:1045D000F6E0EF2EF12CEC0EFD1E0E94E71ED80136
:1045E0008D938D01AE15BF05C1F78B81807380332C
:1045F00009F4A1C000D00F92EDB7FEB711828FEC85
:1046000098E0938382830E94391115E00F900F90F8
:104610000F9050C00E94E31E1092B80600D00F9277
:10462000ADB7BEB711961C92119780E098E0139633
:104630009C938E9312970E94391111E00F900F9066
:104640000F90812F26960FB6F894DEBF0FBECDBF18
:10465000CF91DF911F910F91FF90EF90DF90CF905E
:10466000089582E08093B9068E010E5F1F4FA6E089
:10467000EA2EF12CEC0EFD1E0E94E71EF80181933C
:104680008F01EE15FF05C1F78D818A3AB1F000D098
:104690000F92ADB7BEB711961C92119780E399E0C7
:1046A00013969C938E9312970E94391114E00F90E9
:1046B0000F900F900E94F31EC4CF8C818F708130B9
:1046C00009F476CF00D00F92EDB7FEB7118280E1EA
:1046D00099E0938382830E94391115E00F900F9027
:1046E0000F90E8CF00D000D00F92EDB7FEB7319613
:1046F000ADB7BEB711961C928DE499E09283818389
:10470000238314820E94391114E00F900F900F90B0
:104710000F900F90CFCF00D00F92EDB7FEB7118260
:104720008DEE98E0938382830E94391116E00F90FA
:104730000F900F90BFCF80ED97E00E94ED147C01A9
:1047400089E240E050E060E070E00E944322182FD0
:1047500087FD54C0C7010E94F714882309F081C067
:1047600010FDEECF112389F100D00F92ADB7BEB787
:1047700011961C92119781EA98E013969C938E9360
:1047800012970E94391113E00F900F900F9092CF63
:1047900000D000D00F92EDB7FEB73196ADB7BEB7DF
:1047A00011961C928DEF98E0A9CF00D00F92EDB733
:1047B000FEB711828FE599E0938382830E943911BD
:1047C00012E00F900F900F9075CF80E140E052E023
:1047D00060E070E00E947720882349F100D00F92BA
:1047E000EDB7FEB711828EE798E0938382830E9433
:1047F00039111BE00F900F900F905CCF00D000D0CC
:104800000F92EDB7FEB73196ADB7BEB711961C92B9
:104810008BEB98E092838183138314820E94391179
:1048200014E00F900F900F900F900F9043CF8EEBEE
:1048300096E00E942D22182F882319F100D00F92A4
:10484000ADB7BEB711961C92119789E698E0139602
:104850009C938E9312970E9439110F900F900F9096
:1048600029CF00D00F92EDB7FEB711828DEA98E004
:10487000938382830E94391113E00F900F900F9061
:1048800019CF8EEC96E00E941722182F882379F01A
:1048900000D00F92EDB7FEB7118286E598E09383C2
:1048A00082830E9439110F900F900F9003CF00D098
:1048B0000F92ADB7BEB711961C92119781E598E0A3
:1048C00013969C938E9312970E9439118091CE0675
:1048D0000F900F900F90829586958695837009F4BE
:1048E0008AC0813009F45FC01092BA061092BB06EC
:1048F0001092BC061092BD068091B906813009F471
:104900003FC0823071F400D00F92EDB7FEB7118234
:1049100086E298E0938382830E9439110F900F9072
:104920000F908091BA069091BB06A091BC06B09101
:10493000BD0600D000D00F924DB75EB74F5F5F4FFE
:10494000EDB7FEB7118221E138E0FA01328321830D
:1049500004E1B695A795979587950A95D1F7948325
:1049600083830E9439110F900F900F900F900F903A
:104970008EEB96E00E94511F81E08093B8069ACE9C
:1049800000D00F92ADB7BEB711961C92119780E47C
:1049900098E013969C938E9312970E9439110F9072
:1049A0000F900F90BECF8091D5068091D6062091B2
:1049B000D70690E0A0E0B0E0BA2FA92F982F882763
:1049C00030E040E050E0822B932BA42BB52B23E169
:1049D000880F991FAA1FBB1F2A95D1F780509040BE
:1049E000A84FBF4F8093BA069093BB06A093BC0616
:1049F000B093BD0681CF6091D3068091D406C82EB6
:104A0000DD24EE24FF2483E090E0A0E0B0E0C822A3
:104A1000D922EA22FB22EAE0CC0CDD1CEE1CFF1CB2
:104A2000EA95D1F72091D5068091D6068295869594
:104A30008695837090E0A0E0B0E030E040E050E088
:104A4000220F331F441F551F220F331F441F551FB2
:104A5000822B932BA42BB52B2091D7064091D806FF
:104A60002370220F441F4427441F242B8C299D2987
:104A7000AE29BF290196A11DB11D30E02E5F3F4F29
:104A800004C0880F991FAA1FBB1F2A95D2F76F7009
:104A900004C0880F991FAA1FBB1F6A95D2F7809385
:104AA000BA069093BB06A093BC06B093BD0624CF74
:104AB000FC01009709F475C08185882309F471C051
:104AC0008281282F30E040E050E02F70307040703D
:104AD0005070A5E1220F331F441F551FAA95D1F72F
:104AE000808191818C5B9740A0E0B0E079E1880FF4
:104AF000991FAA1FBB1F7A95D1F7282B392B4A2B58
:104B00005B2B838190E0A0E0B0E08F719070A0708B
:104B1000B070DC0199278827282B392B4A2B5B2B77
:104B2000848190E0A0E0B0E07BE0880F991FAA1F8D
:104B3000BB1F7A95D1F7A070B070282B392B4A2B68
:104B40005B2B858190E0A0E0B0E08F739070A07047
:104B5000B070880F991FAA1FBB1F880F991FAA1F2B
:104B6000BB1F880F991FAA1FBB1F880F991FAA1F61
:104B7000BB1F880F991FAA1FBB1F282B392B4A2B3D
:104B80005B2B8681869590E0A0E0B0E08F719070FD
:104B9000A070B070282B392B4A2B5B2BB901CA01AE
:104BA000089520E030E040E050E0B901CA010895E6
:104BB00080911409882361F08091340B882319F1C6
:104BC0008091540D882319F140E050E0CA01089506
:104BD00060E070E090E020E232E0829FA001839FDD
:104BE000500D929F500D11244B50594F629FF00170
:104BF000639FF00D729FF00D1124EC5EF64F81E083
:104C00008083CA01089581E061E070E0E3CF82E033
:104C100062E070E0DFCFFC01009761F086E0E53FE5
:104C2000F80751F089E0E531F80731F08BE0E53322
:104C3000F80711F080E00895E15EFD4F1082EF511A
:104C4000F24010821182128213821482158216821F
:104C5000178210861286118613861486158616868C
:104C60001786108A118A128A138AE55EFD4F108218
:104C7000118212821382EB51F240148A158A168A2D
:104C8000178A118E108E128E81E008950F931F9354
:104C9000CF93DF93EC0120E088818F3209F45DC06F
:104CA000DE01A20FB11D8C91882349F08F3239F0BB
:104CB0002F5FDE01A20FB11D8C918823B9F78D0102
:104CC0001097B1F3FB01138620E030E080E2FB0196
:104CD000E20FF31F80832F5F3F4F2B303105B9F771
:104CE00090E088818F32B9F1392F3F5F40E0315039
:104CF000FE01E30FF11D3F5FEA17FB07C0F44B30E5
:104D000010F520812E3259F1822F81568A31A8F474
:104D1000FB01E40FF11D205220834F5F3F5F3150B4
:104D2000FE01E30FF11D3F5FEA17FB0740F3C801E7
:104D3000DF91CF911F910F910895FB01E40FF11DB9
:104D400020834F5FEBCF00E010E0C801DF91CF91EF
:104D50001F910F91089591E0C7CF21E0A1CF493075
:104D600090F748E03F5FDBCF9C018091DE0688230F
:104D700009F12230310528F18091DF0690E02250C0
:104D80003040AC01249FC001259F900D349F900DB1
:104D90001124A0E0B0E02091ED063091EE064091A4
:104DA000EF065091F006280F391F4A1F5B1FB9010B
:104DB000CA01089520E030E040E050E0B901CA01A6
:104DC000089580E090E0A0E0B0E0E5CFEF92FF92A0
:104DD0000F931F937B018C018091DE068823E9F0FD
:104DE0008091ED069091EE06A091EF06B091F0064D
:104DF000E81AF90A0A0B1B0B2091DF0630E040E0AD
:104E000050E0C801B7010E9445442E5F3F4FC901E1
:104E10001F910F91FF90EF90089520E030E0C901BD
:104E20001F910F91FF90EF9008958091DE060895F5
:104E3000FC0160E080899189A289B3890196A11D56
:104E4000B11D248535854685578582179307A407AC
:104E5000B50708F061E0862F08952F923F925F9288
:104E60006F927F928F929F92AF92BF92CF92DF927A
:104E7000EF92FF920F931F93DF93CF93CDB7DEB7DF
:104E8000C050D2400FB6F894DEBF0FBECDBF9C011C
:104E90008091DE06882309F484C0C901A0E0B0E057
:104EA000880F991FAA1FBB1F7C018D0139E0169541
:104EB0000795F794E7943A95D1F72091E50630915C
:104EC000E6064091E7065091E806E20EF31E041F45
:104ED000151F2FEFA22E21E0B22EC12CD12CA8221B
:104EE000B922CA22DB226624772443011E010894DA
:104EF000211C311C08C08FEF91E0A0E0B0E0A82297
:104F0000B922CA22DB22E614F7040805190551F07C
:104F1000C801B701A1010E94FA21882309F041C00C
:104F200037014801F101EA0DFB1D20813181552433
:104F3000C90102978E5E9F4F10F45524539411823D
:104F400010825901CC24DD24AA0CBB1CCC1CDD1C16
:104F500086017501B9E016950795F794E794BA951F
:104F6000D1F78091E5069091E606A091E706B09111
:104F7000E806E80EF91E0A1F1B1FE614F7040805D1
:104F8000190519F4552009F0B6CFC401B301A101E8
:104F90000E94D620882329F4552009F0ACCF81E067
:104FA00001C080E0C050DE4F0FB6F894DEBF0FBEE8
:104FB000CDBFCF91DF911F910F91FF90EF90DF90C8
:104FC000CF90BF90AF909F908F907F906F905F90A9
:104FD0003F902F9008950F931F93CF93DF93C5EFCA
:104FE000D6E000E010E0C15EDD4F8881CF51D240B5
:104FF000813081F0C05EDD4F8DE0C535D80799F76F
:105000000E94251F1092DE06802FDF91CF911F9105
:105010000F910895CE010E949528080F191FEACF1D
:10502000CF92DF92EF92FF920F931F93CF93DF9374
:10503000EC01009761F42FEF3FEFC901DF91CF91B1
:105040001F910F91FF90EF90DF90CF900895809186
:10505000DE06882381F38B85813611F0873759F777
:1050600089859A85892B09F045C0BBE1CB2EB2E03A
:10507000DB2ECC0EDD1EABE1EA2EF12CEC0EFD1E7C
:105080006C897D898E899F89F60160837183828313
:105090009383A7010E94FA21882309F041C0088D5B
:1050A000198D000F111F02951295107F1027007F98
:1050B00010270E0D1F1D8C859D85AE85BF85F801BF
:1050C000848F958FA68FB78F8EE996E00E94582522
:1050D000F801668B778B808F918FF60160817181EB
:1050E00082819381A7010E94D6208823C9F420E001
:1050F00030E0A3CFFBE1CF2EF2E0DF2ECC0EDD1EA1
:10510000F6016081718182819381EBE1EE2EF12CB9
:10511000EC0EFD1EA7010E94D620882309F4B0CF13
:105120000E94EB272FEF3FEF88CF0F931F93CF9372
:10513000DF93EC01009761F00E9410288C01CE01F2
:105140000E940B26C801DF91CF911F910F91089506
:105150000FEF1FEFC801DF91CF911F910F910895BD
:105160004F925F926F927F928F929F92AF92BF9277
:10517000CF92DF92EF92FF920F931F93CF93DF9323
:10518000BC018091DE06882309F441C061157105D8
:10519000F1F14BE1C42ED12CC60ED71E88249924E0
:1051A0005401EE24FF2487013BE1632E32E0732E8D
:1051B000660E771E44244A94542C6091E506709143
:1051C000E6068091E7069091E806680D791D8A1D34
:1051D0009B1DD3016D937D938D939C931397A60193
:1051E0000E94FA21882309F058C0F601C0E0D0E0FF
:1051F00080819181892BF9F02196329681E0C0302F
:10520000D807B1F720E030E040E050E02AC040E0AD
:1052100050E0CA01DF91CF911F910F91FF90EF9065
:10522000DF90CF90BF90AF909F908F907F906F90C6
:105230005F904F90089551824082F30160817181A7
:1052400082819381A6010E94D620882331F5D8015E
:10525000C701B695A795979587959E01280F391F89
:10526000A9010894811C911CA11CB11C8091E3062A
:105270009091E406A0E0B0E088169906AA06BB0665
:1052800040F680E092E0A0E0B0E0E80EF91E0A1FD0
:105290001B1F232B09F491CFBCCF0E94EB2740E0CA
:1052A00050E0B7CF8F929F92AF92BF92CF92DF9292
:1052B000EF92FF920F931F93CF93DF938C01809116
:1052C000DE06882321F10115110509F1D801149694
:1052D0002D913D914D915C9117978091ED069091A4
:1052E000EE06A091EF06B091F006281739074A079D
:1052F0005B0768F08091F1069091F206A091F306A9
:10530000B091F40682179307A407B50780F4C0E0B4
:10531000D0E0CE01DF91CF911F910F91FF90EF90E0
:10532000DF90CF90BF90AF909F908F900895CA016B
:10533000B9010E94E626EC014C01AA24BB24880C8A
:10534000991CAA1CBB1C7501640159E0F694E794F2
:10535000D794C7945A95D1F78091E5069091E606C7
:10536000A091E706B091E806C80ED91EEA1EFB1E02
:10537000F801E55EFD4F80819181A281B3818C159A
:105380009D05AE05BF0581F0C082D182E282F38225
:10539000A801455E5F4FC701B6010E94FA2188232C
:1053A00019F00E94EB27B5CF8FEF91E0A0E0B0E0BD
:1053B00088229922AA22BB22F801E80DF91DC38D8B
:1053C000D48D9FEFC83FD90708F0A1CFCE010E942E
:1053D000B426D80114966D937D938D939C93179763
:1053E00018961C9218971A961C921E92199791CF94
:1053F000CF92DF92EF92FF920F931F93CF93DF93A1
:10540000EC017A018B018091DE06882309F456C0F5
:10541000209709F453C02115310509F069C040E017
:1054200050E060E070E0E40EF51E061F171F17FD48
:1054300051C08C859D85AE85BF858E159F05A007C3
:10544000B1070CF447C088819981AA81BB818C8304
:105450009D83AE83BF8318861A861986188A198A97
:105460001A8A1B8AC12C72E0D72E6091DF06288928
:1054700039894A895B892E153F054007510770F528
:105480002F5F3F4F4F4F5F4F288B398B4A8B5B8B82
:1054900089859A8501969A8789878050924038F34A
:1054A0001A86198688858F5F8887861700F3CE0154
:1054B0000E945229892B49F11886D7CF60E070E00D
:1054C000CB01DF91CF911F910F91FF90EF90DF9073
:1054D000CF900895288939894A895B8960E070E016
:1054E000E216F3060407150759F361E070E0E8CF10
:1054F0002230310529F0488959896A897B8993CFFF
:105500004C855D856E857F858ECF888581508887A7
:10551000DA86C986AACFCF92DF92EF92FF920F93DD
:105520001F93CF93DF938C018091DE06882361F473
:10553000CFEFDFEFCE01DF91CF911F910F91FF9061
:10554000EF90DF90CF9008950115110589F3F801D0
:1055500084859585A685B7850097A105B10541F39A
:1055600040895189628973894F5F5F4F6F4F7F4FC9
:10557000481759076A077B07D8F6C480D580E680AC
:10558000F7808085C80ED11CE11CF11CE55EFD4F43
:1055900080819181A281B3818C159D05AE05BF05E7
:1055A000B1F0C082D182E282F382A801455E5F4FF2
:1055B000C701B6010E94FA218823C9F5F801408984
:1055C0005189628973894F5F5F4F6F4F7F4FF80139
:1055D00081859285E80FF91F238DC22FD0E0F80155
:1055E000408B518B628B738B0196928781878050A1
:1055F000924008F49FCFF8011286118680858F5F54
:1056000080879091DF06891708F494CFC8010E9423
:105610005229892B19F0F80110868CCFF80180856A
:105620008150808780E092E09287818783CF0E94BB
:10563000EB27CFEFDFEF7ECFCF92DF92EF92FF929B
:105640000F931F93CF93DF93EC018A018091DE06C5
:10565000882361F4C0E0D0E0CE01DF91CF911F91AB
:105660000F91FF90EF90DF90CF9008954115510575
:1056700089F3209789F31616170664F761307105D0
:10568000F1F07E016B01C8010E948B2A2FEF8F3F42
:10569000920781F08A30910551F0F70181937F01E3
:1056A0000894C108D108F1E0CF16D10461F7F701E1
:1056B0001082D2CFF7011082C0E0D0E0CDCF7E01C2
:1056C000F6CF4F925F926F927F928F929F92AF929E
:1056D000BF92CF92DF92EF92FF920F931F93CF93DF
:1056E000DF93FC015A016B012801390147018091C8
:1056F000DE06882389F1E114F10471F1309761F13C
:10570000011511052105310539F1EF01EE24FF24C2
:105710008701A114B104C104D104A1F0C4010E9405
:105720008B2A2FEF8F3F920769F580E0E414F50490
:1057300006051705A0F4882391F0A114B104C10453
:10574000D10461F70894E11CF11C011D111D81E0D9
:10575000AA24BB246501EACFEE24FF248701B70108
:10576000C801DF91CF911F910F91FF90EF90DF90D3
:10577000CF90BF90AF909F908F907F906F905F90F1
:105780004F90089589930894A108B108C108D108E1
:10579000C0CF2F923F924F925F926F927F928F92E3
:1057A0009F92AF92BF92CF92DF92EF92FF920F93B0
:1057B0001F93DF93CF93CDB7DEB72C970FB6F89436
:1057C000DEBF0FBECDBF98878F8369874A873901B7
:1057D0008091DE06882309F420C12115310509F4E2
:1057E0001CC1EF80F884EF2809F417C1D9011D927C
:1057F0001D921D921C92139754962D913D914D919F
:105800005C915797211531054105510509F0EAC012
:105810008091E1069091E206880F991F82959295FA
:10582000907F9827807F9827892F992786957C01DC
:1058300000E010E0EB82FC820D831E838091E9067C
:105840009091EA06A091EB06B091EC06F3018083FB
:105850009183A283B3830097A105B10509F423C105
:10586000EBE12E2EE2E03E2E260C371C7BE1472E8C
:10587000512C460C571CF30180819181A281B38188
:1058800084839583A683B7831086128611861A8235
:105890001982882499245401D3011496CD90DD9067
:1058A000ED90FC901797C80CD91CEA1CFB1CF10169
:1058B000C082D182E282F382C701B601A2010E94B6
:1058C000FA21882309F043C15C864B8600E010E092
:1058D0000CC00F5F1F4F2B853C85205E3F4F3C87E0
:1058E0002B870031110509F4B7C0AB85BC859C91AD
:1058F000992379F3953E69F31B963C918A8583231E
:10590000B9858B1731F7AF81B885EB85FC8520E031
:1059100001C090818C91891709F09AC02F5F119670
:1059200031962B30B1F7F301328FAB85BC855A9697
:105930008D919C915B970E94B426F30160837183E3
:1059400082839383D30114966D937D938D939C935F
:10595000179718961C9218971A961C921E921997D0
:10596000C48AD58AE68AF78A118F008FEB85FC8579
:10597000848D958DA68DB78DF30184879587A68735
:10598000B78781E011E00894811C911CA11CB11C17
:105990002B813C814D815E8182169306A406B5065B
:1059A00018F4882309F478CF012F112399F420915A
:1059B000ED063091EE064091EF065091F006F301AE
:1059C00084819581A681B78182179307A407B507C3
:1059D00008F0C1C0E980FA80EF2801F1112309F431
:1059E00058CF1CC08091E9069091EA06A091EB0681
:1059F000B091EC06281739074A075B0780F58091BC
:105A0000ED069091EE06A091EF06B091F0062817F2
:105A100039074A075B0708F081C000E0802F2C9609
:105A20000FB6F894DEBF0FBECDBFCF91DF911F91AF
:105A30000F91FF90EF90DF90CF90BF90AF909F902D
:105A40008F907F906F905F904F903F902F90089530
:105A50002A3008F43ECF67CF80E010E094CF8091E9
:105A6000ED069091EE06A091EF06B091F006281792
:105A700039074A075B0708F051C08091E106909111
:105A8000E206880F991F82959295907F9827807FD4
:105A90009827892F992786957C0100E010E0EB82FA
:105AA000FC820D831E831BE1212E12E0312E260C79
:105AB000371CD1012D933D934D935C931397BBE11C
:105AC0004B2E512C460C571CCA01B901A2010E9451
:105AD000FA218823E1F5D3015896ED91FC9159976D
:105AE000EE0FFF1FE295F295F07FFE27E07FFE2785
:105AF000E40DF51D8081882309F48FCF853E09F4DC
:105B00008CCF838584FF89CF828D938D0E94B426AC
:105B1000F3016083718382839383ADCE8091F1061C
:105B20009091F206A091F306B091F40682179307C4
:105B3000A407B50708F471CF8091DF06E82EFF2493
:105B400000E010E0EB82FC820D831E83ACCF0E944C
:105B5000EB2700E063CFC3010E9452299A83898317
:105B600039CFAF92BF92CF92DF92EF92FF920F9315
:105B70001F93DF93CF93CDB7DEB72C970FB6F89472
:105B8000DEBF0FBECDBFFC01A62EB42E790100975B
:105B9000D1F121153105B9F18091DE06882399F103
:105BA000D90154961D921D921D921C925797599699
:105BB0001C921E9258978081882329F16E010894C7
:105BC000C11CD11C12C060E148E1C60197010E94CE
:105BD000C92B8823C1F090E0D8018C91882309F467
:105BE00091E0892F992381F4F801CF01B6010E9439
:105BF00046268C01009739F0FC018081882319F733
:105C00006A2D4B2DE2CF80E02C960FB6F894DEBFC4
:105C10000FBECDBFCF91DF911F910F91FF90EF90FD
:105C2000DF90CF90BF90AF900895EF92FF920F93C7
:105C30001F938C010E94D8257C01C80160E048E1D7
:105C400097010E94B12D182FC7010E940B26812FAA
:105C50001F910F91FF90EF9008958F929F92AF92B6
:105C6000BF92CF92DF92EF92FF920F931F93CF9349
:105C7000DF938C018091DE06882309F47CC0011536
:105C8000110509F478C0C8010E94B028EC01009702
:105C900009F473C0C80140E050E060E070E022E029
:105CA00030E00E94F829F80164817581868197812E
:105CB0000E94E6266C01EE24FF24CC0CDD1CEE1CB9
:105CC000FF1CA701960179E05695479537952795D2
:105CD0007A95D1F78091E5069091E606A091E706C6
:105CE000B091E806280F391F4A1F5B1F6BE1A62EF3
:105CF00062E0B62EA00EB11EF50160817181828135
:105D00009381621773078407950709F449C0F50169
:105D10002083318342835383BBE18B2E912C800EF1
:105D2000911ECA01B901A4010E94FA21882399F5A4
:105D3000F50160817181828193812FEF31E040E034
:105D400050E0C222D322E422F522F801EC0DFD1D21
:105D5000D48FC38FA4010E94D6208823E1F4CE0102
:105D60000E94B426F8016483758386839783108626
:105D70001286118602C0C0E0D0E0CE01DF91CF9143
:105D80001F910F91FF90EF90DF90CF90BF90AF9059
:105D90009F908F9008950E94EB27C0E0D0E0EDCF58
:105DA0002BE1822E912C800E911EC7CFCF92DF92D5
:105DB000FF920F931F93CF93DF93F82EEB01809107
:105DC000DE06882359F42FEF3FEFC901DF91CF9111
:105DD0001F910F91FF90DF90CF900895611571058D
:105DE00091F3288939894A895B898C859D85AE859F
:105DF000BF85281739074A075B0730F089859A85E0
:105E00008050924008F089C00C811D812E813F8115
:105E10008885080F111D211D311DFBE1CF2EF2E0F9
:105E2000DF2ECC0EDD1EF60180819181A281B3812F
:105E300080179107A207B30771F0008311832283B3
:105E40003383AE01455E5F4FC901B8010E94FA215C
:105E5000882309F05DC069857A85FE01E60FF71F8A
:105E6000F38E8C859D85AE85BF85288939894A89C1
:105E70005B8982179307A407B50781F12F5F3F4F16
:105E80004F4F5F4F288B398B4A8B5B8BCB01019631
:105E90009A8789878050924018F420E030E095CFAF
:105EA000F6016081718182819381AE01455E5F4F11
:105EB0000E94D620882361F51A86198688858F5F0F
:105EC00088879091DF06891740F3CE010E945229FE
:105ED000892B79F0188620E030E077CF9C01AD0166
:105EE0002F5F3F4F4F4F5F4F2C873D874E875F8718
:105EF000C9CFCE010E942D2E892B79F6888581503D
:105F0000888780E092E09A8789872FEF3FEF5DCF07
:105F10000E94EB272FEF3FEF58CFCB010E942D2E91
:105F2000892B09F071CF4FCFEF92FF921F93CF9340
:105F3000DF93EC017B018091DE06882301F161157E
:105F40007105E9F02097D9F088818823C1F010E02D
:105F500004C09FEF2F3F3907A1F0B7010E94D62E52
:105F60009C011F5FFE01E10FF11D8081882389F7ED
:105F7000C901DF91CF911F91FF90EF90089520E02C
:105F800030E0C901DF91CF911F91FF90EF9008950C
:105F90004F925F926F927F928F929F92AF92BF9239
:105FA000CF92DF92EF92FF920F931F93CF93DF93E5
:105FB000FC015A016B012801390147018091DE067D
:105FC000882389F1E114F10471F1309761F1011531
:105FD00011052105310539F1EF01EE24FF24870178
:105FE000A114B104C104D104A1F08881B4010E94BC
:105FF000D62E8F5F9F4F69F580E0E414F504060507
:106000001705A0F4882391F0A114B104C104D104B0
:1060100061F70894E11CF11C011D111D81E0AA2407
:10602000BB246501EACFEE24FF248701B701C80134
:10603000DF91CF911F910F91FF90EF90DF90CF9064
:10604000BF90AF909F908F907F906F905F904F9098
:10605000089521960894A108B108C108D108C0CFBD
:106060009F92AF92BF92CF92DF92EF92FF920F93E7
:106070001F93CF93DF93EC018091DE06882309F410
:1060800051C0209709F44EC080E090E0A0E0B0E05D
:10609000FE01E81BF90B138E0197A109B1098030AD
:1060A0002EEF92072FEFA2072FEFB20789F780910B
:1060B000DF06882309F444C0BBE1AB2EB12CAC0E43
:1060C000BD1E99249394EE24FF248701ABE1CA2ED0
:1060D000A2E0DA2ECC0EDD1E0FC00894E11CF11CEC
:1060E000011D111D8091DF0690E0A0E0B0E0E816F0
:1060F000F9060A071B07B8F46C817D818E819F81A8
:106100006E0D7F1D801F911FF60160837183828356
:106110009383A5010E94D6208823F9F20E94EB27E1
:106120009924DBCF9924892DDF91CF911F910F9175
:10613000FF90EF90DF90CF90BF90AF909F90089529
:1061400099249394F0CF2F923F924F925F926F9247
:106150007F928F929F92AF92BF92CF92DF92EF92F7
:10616000FF920F931F93DF93CF93CDB7DEB7639763
:106170000FB6F894DEBF0FBECDBF2C016D878A012C
:106180008091DE06882309F4C6C04115510509F443
:10619000C2C04114510409F4BEC0DA011D921D921F
:1061A0001D921C92139754962D913D914D915C91A7
:1061B0005797211531054105510509F091C080918E
:1061C000E1069091E206880F991F82959295907F43
:1061D0009827807F9827892F992786955C01CC2462
:1061E000DD24AD82BE82CF82D8868091E90690916F
:1061F000EA06A091EB06B091EC06F801808391834A
:10620000A283B3830097A105B10509F4C3C01C8222
:106210001B82C8010E94B0281C01009709F47BC0B2
:10622000F80180819181A281B38184839583A683C3
:10623000B78310864BE1842E912C800E911E3BE398
:10624000632E712C600E711E1A8219829801255ED0
:106250003D4F3F872E875D85452F50E04071507040
:10626000598B488B19861A861B861C86D801149672
:10627000AD90BD90CD90DC90179729853A854B85E0
:106280005C85A20EB31EC41ED51EAE85BF85AD9221
:10629000BD92CD92DC921397C601B501A4010E9474
:1062A000FA21882309F0D1C19B8A8A8AEE24FF242F
:1062B000EA89FB898081882309F4C3C0853E09F4FB
:1062C000C0C00894E11CF11CEA89FB89B096FB8BE5
:1062D000EA8BF0E1EF16F10459F780E0FF2416C1D4
:1062E0008091E9069091EA06A091EB06B091EC0648
:1062F000281739074A075B0748F58091ED0690910A
:10630000EE06A091EF06B091F006281739074A076C
:106310005B0708F07DC0FF248F2D63960FB6F894BD
:10632000DEBF0FBECDBFCF91DF911F910F91FF90C8
:10633000EF90DF90CF90BF90AF909F908F907F9025
:106340006F905F904F903F902F9008958091ED0651
:106350009091EE06A091EF06B091F006281739074C
:106360004A075B0708F054C08091E1069091E2066D
:10637000880F991F82959295907F9827807F982704
:10638000892F992786955C01CC24DD24AD82BE82BD
:10639000CF82D886055E1D4FD8012D933D934D9336
:1063A0005C9313970B5112406BE1E62EF12CE00E3B
:1063B000F11ECA01B901A7010E94FA21882309F040
:1063C00044C1D8015896ED91FC915997EE0FFF1FEB
:1063D000E295F295F07FFE27E07FFE27EE0DFF1D90
:1063E0008081882309F497CF853E09F494CF838573
:1063F00084FF91CFA28CB38CBC82AB82C5010E947A
:10640000B426D8016D937D938D939C93139701CF00
:106410008091F1069091F206A091F306B091F406F6
:1064200082179307A407B50708F475CF8091DF069C
:10643000C82EDD24EE24FF24CD82DE82EF82F88692
:10644000A9CF20E030E0EA89FB89E20FF31FD201F7
:10645000A20FB31F8C9180832F5F3F4F2B303105EC
:1064600091F7ED85AA89BB891B96EC931B975B96E8
:106470003C922E925A978EE996E00E945825AA895E
:10648000BB8956966D937D938D939C935997FD018F
:10649000148E158E168E178EAE85BF856D917D91EB
:1064A0008D919C91A4010E94D620882309F0CDC033
:1064B000C1010E94B426F8016083718382839383B3
:1064C000D80114966D937D938D939C93179718968E
:1064D0001C9218971A961C921E921997ED855A963F
:1064E000EC935A971C961D921D921D921C921F9719
:1064F000F801A48AB58AC68AD78AF18EE08EA88868
:10650000B988AB28E9F581E0FF24F39429853A8521
:106510004B855C852F5F3F4F4F4F5F4F29873A87F1
:106520004B875C87AD80BE80CF80D8842A153B0521
:106530004C055D0518F4882309F498CEFF20B9F4C2
:106540002091ED063091EE064091EF065091F00655
:10655000F80184819581A681B78182179307A407EA
:10656000B50728F0C8010E9452299A838983A9801F
:10657000BA80AB2809F4D0CEFF2009F473CECCCE7C
:10658000C8010E943030D8016D917D918D919C9110
:10659000EE85FF856083718382839383A4010E94CB
:1065A000FA21882309F051C0EEE2D401EC93F40102
:1065B00081E020E2A22EA1828F5F31968B30C9F755
:1065C000E0E1D4011B96EC931B975B963C922E92D4
:1065D0005A9756961D921D921D921C925997F4013E
:1065E000148E158E168E178EEEE2D301EC93FEE21A
:1065F0001196FC93F30182E090E2A92EA2828F5FB4
:1066000031968B30C9F7E0E1D3011B96EC931B97D1
:10661000AB80BC805B96BC92AE925A9756961D9208
:106620001D921D921C925997F301148E158E168E91
:10663000178EAE85BF856D917D918D919C91A40142
:106640000E94D620882309F45ECF0E94EB27FF2406
:1066500063CE9F92AF92BF92CF92DF92EF92FF9262
:106660000F931F93DF93CF93CDB7DEB72C970FB661
:10667000F894DEBF0FBECDBF9C01962E6A01009735
:10668000B1F14115510599F18091DE06882379F128
:10669000F901DA0154961D921D921D921C92579792
:1066A00059961C921E9258978081EE245E010894A0
:1066B000A11CB11C8823E1F0EE20D1F4CF01B5017B
:1066C0000E9446268C01009799F0FC018081882366
:1066D000B1F1B0E1FB2EC5016F2D48E196010E949A
:1066E000C92B8823C1F0D8018C91F801E3CFEE24A7
:1066F0008E2D2C960FB6F894DEBF0FBECDBFCF9176
:10670000DF911F910F91FF90EF90DF90CF90BF909E
:10671000AF909F900895F8018081882309F4F92CA7
:10672000C5016F2DA6010E94A330882309F3D8016B
:106730008C918823D1F6EE24E394F801BBCFFF249B
:10674000CACFFF920F931F93CF93DF938C01F62E46
:106750008091DE06882349F4C0E0D0E0CE01DF91CD
:10676000CF911F910F91FF90089501151105A1F38D
:106770000E94D825EC01009789F3188219821A82A9
:106780001B821C821D821E821F8218861A86198611
:10679000FB861C861D861E861F86188A198A1A8A01
:1067A0001B8AC55EDD4F188219821A821B82CB516B
:1067B000D2401C8A1D8A1E8A1F8A198E188E1A8E34
:1067C000C80160E048E19E010E94B12D882381F05C
:1067D00082E7F81609F455C087E7F81629F181E633
:1067E000F816A9F0CE010E949528C0E0D0E0B6CFFF
:1067F00081E6F81619F087E7F816A1F7C80160E2FC
:10680000AE010E942933882309F0A8CFEBCF8A8DEF
:1068100080FDE8CFCE0140E050E060E070E022E093
:1068200030E00E94F8299ACF8A8D80FDDBCF688105
:1068300079818A819B810E94E6260E942D27CE01C4
:106840000E94B0280E94B426688379838A839B8340
:106850006C837D838E839F8318861A8619861C8697
:106860001D861E861F86188A198A1A8A1B8ACE01DF
:1068700040E050E060E070E020E030E00E94F82965
:106880006DCFCE0140E050E060E070E020E030E00D
:106890000E94F82963CF8F929F92AF92BF92CF92BE
:1068A000DF92EF92FF920F931F9300D00F92EDB7FC
:1068B000FEB7118286E09BE0938382830E943911A8
:1068C0001092DE06109214091092340B1092540D9F
:1068D0000F900F900F900E945F228823E9F000D064
:1068E0000F92EDB7FEB7118284EE9AE09383828314
:1068F0000E94391111E00F900F900F900E94EB272A
:10690000812F1F910F91FF90EF90DF90CF90BF905C
:10691000AF909F908F90089560E070E080E090E0ED
:1069200040E157E00E94FA21882319F58091D208AE
:10693000843079F1863069F18E3059F188249924B8
:10694000540180911B0790911C078050924009F4DC
:1069500040C000D00F92EDB7FEB7118286E99AE0F1
:10696000938382830E94391114E00F900F900F904F
:10697000C5CF00D00F92EDB7FEB711828DEC9AE033
:10698000938382830E94391112E00F900F900F9031
:10699000B5CF8090D6089090D708A090D808B09036
:1069A000D908C501B40140E157E00E94FA218823CB
:1069B00041F200D00F92EDB7FEB7118286EB9AE05C
:1069C000938382830E94391113E00F900F900F90F0
:1069D00095CF80911D078093DF066091200760931B
:1069E000E006C0902107D0902207D092E206C09224
:1069F000E10620912607309127073093E406209383
:106A0000E306E0901E07F0901F0700E010E0E80C9E
:106A1000F91C0A1D1B1DE092E506F092E6060093A4
:106A2000E7061093E80670E080E090E040E050E078
:106A30000E94FF436E0D7F1D801F911F6093E9062A
:106A40007093EA068093EB069093EC06D294C2947E
:106A50001FE0C122CD24D122CD24960140E050E098
:106A6000260F371F481F591F2093ED063093EE065F
:106A70004093EF065093F0068091300790913107D4
:106A8000A0913207B09133070097A105B10519F124
:106A90000197A109B109820F931FA41FB51F80930D
:106AA000F1069093F206A093F306B093F40680915A
:106AB0004607863401F100D00F92EDB7FEB7118280
:106AC00087E59AE0938382830E94391116E00F9044
:106AD0000F900F9013CF00D00F92EDB7FEB7118239
:106AE0008AE79AE0938382830E94391115E00F9020
:106AF0000F900F9003CF809147078134E1F680918A
:106B000048078435C1F6809149078133A1F6809109
:106B10004A07863381F681E08093DE0600D00F922B
:106B2000EDB7FEB7118280E59AE0938382830E94DD
:106B3000391110E00F900F900F90E2CECF93DF93BA
:106B4000FC01EB01009731F06115710519F08485A6
:106B5000882321F480E0DF91CF9108958081918195
:106B6000A281B38188839983AA83BB838481958121
:106B7000A681B7818C839D83AE83BF8380859185F9
:106B8000A285B38588879987AA87BB8781E08C8790
:106B9000DF91CF910895FC01009779F01082118266
:106BA0001282138214821582168217821086118631
:106BB00012861386148681E0089580E00895CF93AD
:106BC000DF9380916D04813081F1813040F082301B
:106BD00009F470C010926D04DF91CF9108958091F7
:106BE000A6039091A70381609093A7038093A603C7
:106BF00010929005109291051092920510929305B3
:106C00001092940510929505109296051092970592
:106C1000109298051092990510929A0510929B0572
:106C200010929C05DF91CF91089588EE93E00E9429
:106C3000ED1490938404809383048091A603909133
:106C4000A7038E7F9093A7038093A603C09181042E
:106C5000D09182042196D0938204C09381048091C4
:106C6000500490E083709070892B81F5109290050C
:106C7000109291051092920510929305109294052E
:106C8000109295051092960510929705109298050E
:106C90001092990510929A0510929B0510929C05EE
:106CA0008091A8038230E9F082E080936D04DF9147
:106CB000CF91089580918304909184040E94F714E9
:106CC000882309F087CFDF91CF91089580914F04F9
:106CD000843060F281E494E060E975E00E949E35C2
:106CE000DFCF80914E0480FD0EC0CE0165E070E0E4
:106CF0000E941E44892B39F484E690E09093C303EC
:106D00008093C203D1CF80914F04843068F6CE01C6
:106D100065E070E00E941E44892B31F68AE090E025
:106D20009093C3038093C203BFCF809104029091DC
:106D30000502909303028093020280911F029091BA
:106D4000200290931E0280931D020895982FDB016C
:106D50008091EF01891731F080910A028917D1F0F3
:106D600080E0089580E090E0FC01EE0FFF1FE80F47
:106D7000F91FCF01880F991F880F991F880F991F3E
:106D8000E80FF91FE151FE4F838994898D939C93FD
:106D900081E0089581E090E0E7CFCF92DF92EF921B
:106DA000FF920F931F93DF93CF93CDB7DEB7629718
:106DB0000FB6F894DEBF0FBECDBF9C018B010097CC
:106DC00009F44BC06115710509F447C07E010894B0
:106DD000E11CF11CD701E1ECF1E082E101900D92A0
:106DE0008150E1F7F90101900020E9F731974E2F2A
:106DF000421B413108F040E1C701B90150E00E9457
:106E0000B644C70160EF71E040E150E00E94BF442A
:106E1000009799F1C7016BE072E040E150E00E94F9
:106E2000BF44009709F48EC000D000D00F92EDB798
:106E3000FEB73196ADB7BEB711961C9288EA9BE0BB
:106E400092838183F482E3820E94391180E00F9063
:106E50000F900F900F900F9001C080E062960FB6D8
:106E6000F894DEBF0FBECDBFCF91DF911F910F9180
:106E7000FF90EF90DF90CF900895CC24DD24C801DF
:106E80000E9482449C01B601660F771FCB018C0DD6
:106E90009D1DFC01EE0FFF1FEE0FFF1FEE0FFF1FEA
:106EA000E80FF91FE151FE4F348B238B4789508D3A
:106EB0002417350738F0818D928D8217930710F0D3
:106EC00081E0CCCF8DB79EB70B970FB6F8949EBFDD
:106ED0000FBE8DBFEDB7FEB73196ADB7BEB71196F9
:106EE0001C9285EC9BE092838183F482E38236835B
:106EF000258350874783CB018C0D9D1D8C01000F8E
:106F0000111F000F111F000F111F080F191F015132
:106F10001E4FD80159968D919C915A9792878187DF
:106F20000E943911F80185899689948B838B81E0C1
:106F30002DB73EB7255F3F4F0FB6F8943EBF0FBE4B
:106F40002DBF8CCFF1E0CF2ED12C99CFAF92BF9235
:106F5000CF92DF92EF92FF920F931F93DF93CF9325
:106F6000CDB7DEB7A2970FB6F894DEBF0FBECDBF88
:106F700000D00F92ADB7BEB711961C92119784E95D
:106F80009BE013969C938E9312970E9439118091E7
:106F90000402909105029093030280930202809173
:106FA0001F029091200290931E0280931D020F9069
:106FB0000F900F900E941527882309F445C083ED98
:106FC00091E00E94152E882309F45DC083ED91E0C5
:106FD00062E70E94A1338C01009709F4FCC083E0B2
:106FE000A82EB12CAC0EBD1E7E010894E11CF11C34
:106FF000C50160E270E0A8010E941C2B892B09F4F6
:10700000C5C08B818A30A1F38D3091F3803281F33A
:107010008B3371F3833261F3C50160EE71E0A70138
:107020000E94CD446C0180E090E060EE71E0A70129
:107030000E94CD44BC01C114D104D1F20097C1F229
:10704000C6010E94CD36D4CF00D00F92EDB7FEB767
:10705000118287E19BE0938382830E9439110F9014
:107060000F900F90A2960FB6F894DEBF0FBECDBF63
:10707000CF91DF911F910F91FF90EF90DF90CF9014
:10708000BF90AF90089583ED91E067E70E94A13330
:107090005C01009709F490C0B3E0EB2EF12CEC0EEC
:1070A000FD1E8DB79EB708970FB6F8949EBF0FBE12
:1070B0008DBFEDB7FEB73196ADB7BEB71296FC9255
:1070C000EE921197A2EECA2EA1E0DA2ED382C282EE
:1070D00000EF11E015830483809104029091050272
:1070E000978386830E94FC44EDB7FEB738960FB6AF
:1070F000F894FEBF0FBEEDBFC701B5010E94942FEB
:107100008DB79EB708970FB6F8949EBF0FBE8DBF80
:10711000EDB7FEB73196ADB7BEB71296FC92EE92C0
:107120001197D382C282055E1F4F1583048380911D
:107130001F0290912002978386830E94FC44EDB742
:10714000FEB738960FB6F894FEBF0FBEEDBFC7016D
:10715000B5010E94942F8CEE91E0B5010E94942F0E
:10716000C5010E94952800D00F92ADB7BEB7119609
:107170001C9211978DE29BE013969C938E9312972D
:107180000E9439110F900F900F906CCFC8010E9490
:10719000952800D00F92ADB7BEB711961C921197EB
:1071A00083E79BE013969C938E9312970E9439116C
:1071B0000F900F900F9056CF00D00F92EDB7FEB703
:1071C00011828CE49BE0938382830E9439110F909B
:1071D0000F900F9047CF00D00F92EDB7FEB71182FE
:1071E00086E79BE0938382830E9439110F900F9072
:1071F0000F9038CF0F931F938091A706882309F42F
:107200005BC020919E0630919F0680919C049091D6
:107210009D048217930709F455C05091A0069091E0
:10722000A10630939D0420939C0450939E04909358
:107230009F0481E08093A5041092CA041092C904AF
:10724000492F8DB79EB70C970FB6F8949EBF0FBE0F
:107250008DBFEDB7FEB7319606EA14E0ADB7BEB705
:1072600012961C930E93119785E292E0938382838A
:107270003583248356831782408711868091C90401
:107280009091CA04938782870E94FC448091C9042C
:107290009091CA0401969093CA048093C9049801FE
:1072A0008DB79EB70C960FB6F8949EBF0FBE8DBFDC
:1072B000C9011F910F91089520E030E0C9011F918D
:1072C0000F91089550919E048091A006581721F0C7
:1072D0009091A106582FA5CF40919F049091A106AF
:1072E000491709F09ECFADCFCF93DF93EC01009704
:1072F00001F5809191048330B9F0109291041092BD
:10730000900410928F0488E894E00E94914380E0FA
:1073100090E00E94ED1490938E0480938D048091F0
:107320009104DF91CF91089588E894E00E944A4348
:10733000E4CF80918D0490918E040E94F7148823ED
:1073400031F490919104892FDF91CF910895CE016E
:107350000E94ED1490938E0480938D048091A80375
:107360008230F9F090919104933069F788E894E0C5
:107370000E944A43882309F4A9C000D00F92EDB7B8
:10738000FEB7118286E09CE0938382830E943911CC
:1073900082E0809391040F900F900F9092E0892FDC
:1073A000D3CF90919104923009F459C0933008F0F2
:1073B0004FC0992309F453C0913029F010929104E1
:1073C00090E0892FC1CF0E94FA3890939004809367
:1073D0008F04009709F4B9C00E94152E882399F7ED
:1073E00080918F0490919004009709F4AEC068E8F2
:1073F00074E00E94A143882309F480C080E29EE4E7
:107400000E94ED1490938C0480938B0483E080930E
:10741000910400D000D00F92EDB7FEB73196ADB712
:10742000BEB711961C928DE79CE092838183809178
:107430008F0490919004948383830E9439110F905C
:107440000F900F900F900F9090919104892F7CCF07
:10745000933059F0943009F0B1CF892F75CF81E086
:107460008093910491E0892F6FCF80916D048823E0
:1074700009F469CF80914E0480FF65CF809150045C
:10748000833009F060CF88E894E00E94D7438823D6
:1074900009F070C000D00F92ADB7BEB711961C9224
:1074A00011978BE19CE013969C938E9312970E9408
:1074B00039110F900F900F9088E894E00E944A4392
:1074C00084E08093910494E0892F3ECF00D00F9206
:1074D000ADB7BEB711961C9211978BEE9BE0139639
:1074E0009C938E9312970E94391184E080939104AB
:1074F0000F900F900F9094E0892F26CF84E0809317
:10750000910400D000D00F92EDB7FEB73196ADB721
:10751000BEB711961C928EE59CE092838183809188
:107520008F0490919004948383830E9439110F906B
:107530000F900F900F900F908AE090E00E94ED1452
:1075400090938E0480938D04FCCE84E0809391040C
:1075500000D00F92EDB7FEB7118289E39CE09383D0
:1075600082830E9439110F900F900F909091910497
:10757000892FEACE80918B0490918C040E94F7149D
:10758000882309F4DECE80E29EE40E94ED149093FD
:107590008C0480938B048091890490918A040E94CA
:1075A000102890919104892FCFCE0F931F93809133
:1075B000A706882309F45BC020919E0630919F06A0
:1075C0008091CB049091CC048217930709F455C0A5
:1075D0005091A0069091A1063093CC042093CB0447
:1075E0005093CD049093CE0481E08093D404109204
:1075F000F9041092F804492F8DB79EB70C970FB677
:10760000F8949EBF0FBE8DBFEDB7FEB7319605ED66
:1076100014E0ADB7BEB712961C930E93119786E493
:1076200092E0938382833583248356831782408735
:1076300011868091F8049091F904938782870E94C3
:10764000FC448091F8049091F90401969093F90418
:107650008093F80498018DB79EB70C960FB6F894F6
:107660009EBF0FBE8DBFC9011F910F91089520E0ED
:1076700030E0C9011F910F9108955091CD04809180
:10768000A006581721F09091A106582FA5CF409140
:10769000CE049091A106491709F09ECFADCFCF93AC
:1076A000DF93EC01009701F580919B048330B9F0E2
:1076B00010929B0410929A041092990482E994E02B
:1076C0000E94283D80E090E00E94ED149093980481
:1076D0008093970480919B04DF91CF91089582E974
:1076E00094E00E946C3FE4CF8091970490919804BD
:1076F0000E94F714882331F490919B04892FDF9125
:10770000CF910895CE010E94ED1490939804809338
:1077100097048091A8038230F9F090919B049330F4
:1077200069F782E994E00E946C3F882309F4B7C0AE
:1077300000D00F92EDB7FEB7118281EB9CE09383EE
:1077400082830E94391182E080939B040F900F90F6
:107750000F9092E0892FD3CF90919B04923009F43F
:1077600059C0933008F04FC0992309F453C09130A9
:1077700029F010929B0490E0892FC1CF0E94D53A46
:1077800090939A0480939904009709F4C7C00E94CB
:10779000152E882399F78091990490919A04009767
:1077A00009F4BCC062E974E00E94B33F882309F485
:1077B0008EC080E29EE40E94ED1490939604809324
:1077C000950483E080939B0400D000D00F92EDB726
:1077D000FEB73196ADB7BEB711961C9288E29DE018
:1077E000928381838091990490919A0494838383F6
:1077F0000E9439110F900F900F900F900F90909161
:107800009B04892F7CCF9330C9F0943009F0B1CF1D
:10781000892F75CF80916D04882309F46FCF8091F3
:107820004E0480FF6BCF80915004833009F066CF07
:1078300081E080939B0491E0892F61CF80916D045A
:10784000882309F45BCF80914E0480FF57CF80914D
:107850005004833009F052CF82E994E00E94E83F5F
:10786000882309F070C000D00F92ADB7BEB7119653
:107870001C92119786EC9CE013969C938E93129722
:107880000E9439110F900F900F9082E994E00E94AE
:107890006C3F84E080939B0494E0892F30CF00D02C
:1078A0000F92ADB7BEB711961C92119786E99CE076
:1078B00013969C938E9312970E94391184E08093C3
:1078C0009B040F900F900F9094E0892F18CF84E0C5
:1078D00080939B0400D000D00F92EDB7FEB7319695
:1078E000ADB7BEB711961C9289E09DE0928381836B
:1078F0008091990490919A04948383830E94391112
:107900000F900F900F900F900F908AE090E00E94E0
:10791000ED149093980480939704EECE84E08093C6
:107920009B0400D00F92EDB7FEB7118284EE9CE06D
:10793000938382830E9439110F900F900F90909142
:107940009B04892FDCCE80919504909196040E942F
:10795000F714882309F4D0CE80E29EE40E94ED144F
:10796000909396048093950480919304909194044D
:107970000E94102890919B04892FC1CE0F931F93D2
:1079800007E612E084EF91E090936802809367022B
:1079900080E0B8010E94A63680E090E00E944F3B54
:1079A0000E5F1F4F88EE93E090936A028093690206
:1079B00081E0B8010E94A63680E090E00E94743910
:1079C0001F910F9108951A990895809186049091BE
:1079D00087040E94F7148823B9F38AE090E00E949C
:1079E000ED149093870480938604809185048430FD
:1079F00069F40E9415278823F1F488E893E10E9436
:107A0000ED14909387048093860408958091670213
:107A1000909168020E944F3B80938504843049F323
:107A20008091690290916A020E9474398093850462
:107A30008430F9F208950E94BE3C109285048AE0D9
:107A400090E00E94ED14909387048093860408953B
:107A5000FC0110821282118281E008952F923F92E0
:107A60004F925F926F927F928F929F92AF92BF924E
:107A7000CF92DF92EF92FF920F931F93DF93CF93FA
:107A8000CDB7DEB7E2970FB6F894DEBF0FBECDBF1D
:107A90006C01009721F080914D048823D1F480E09F
:107AA000E2960FB6F894DEBF0FBECDBFCF91DF9147
:107AB0001F910F91FF90EF90DF90CF90BF90AF900C
:107AC0009F908F907F906F905F904F903F902F90FE
:107AD0000895D6018C91833011F711968D919C9168
:107AE0001297892BE1F2E0904104F090420400915A
:107AF00043041091440417FD1FC13BE2832E912CD7
:107B0000C801B70120E836E948E950E00E9467441F
:107B1000562E472E382E292E3E010894611C711CCA
:107B2000EDB7FEB73C970FB6F894FEBF0FBEEDBFA2
:107B3000ADB6BEB60894A11CB11C728261828BE600
:107B400092E0D50113969C938E93129715969C9272
:107B50008E921497C801B70120E836E948E950E051
:107B60000E946744C90137FD03C1F50197838683ED
:107B7000652D742D832D922D20E137E240E050E0F9
:107B80000E946744C90137FDEFC0D50119969C9347
:107B90008E931897652D742D832D922D20E137E259
:107BA00040E050E00E9467442AE030E040E050E0CE
:107BB0000E946744C90137FDD3C0F50193878287CE
:107BC0000E94FC448DB79EB70C960FB6F8949EBFEA
:107BD0000FBE8DBFD60111966D917C911297C30196
:107BE0000E94942FE0904504F090460400914704D1
:107BF0001091480417FDA4C09BE2892E912CC80166
:107C0000B70120E836E948E950E00E946744562E63
:107C1000472E382E292EEDB7FEB73C970FB6F894B5
:107C2000FEBF0FBEEDBFADB6BEB60894A11CB11C21
:107C3000728261828CE792E0D50113969C938E93B9
:107C4000129715969C928E921497C801B70120E85E
:107C500036E948E950E00E946744C90137FD78C021
:107C6000F50197838683652D742D832D922D20E158
:107C700037E240E050E00E946744C90137FD64C02C
:107C8000D50119969C938E931897652D742D832D8D
:107C9000922D20E137E240E050E00E9467442AE064
:107CA00030E040E050E00E946744C90137FD54C015
:107CB000F501938782870E94FC448DB79EB70C968E
:107CC0000FB6F8949EBF0FBE8DBFD60111966D9171
:107CD0007C911297C3010E94942FEDB7FEB73A979B
:107CE0000FB6F894FEBF0FBEEDBF3196ADB7BEB76D
:107CF00012967C926E9211978BE892E09383828326
:107D00008BE290E095838483178216821186108619
:107D10000E94FC44EDB7FEB73A960FB6F894FEBF4A
:107D20000FBEEDBFD60111966D917C911297C301E4
:107D30000E94942F81E0B4CE2DE2822E912CE0CED1
:107D40008DE2882E912C5BCF909581959F4F98CF97
:107D5000909581959F4F84CF909581959F4FA8CF07
:107D6000909581959F4F29CF909581959F4F0DCFED
:107D7000909581959F4FF9CE0F931F93CF93DF93EB
:107D80008C01FC018081833031F080E0DF91CF9164
:107D90001F910F9108956181728161157105A9F399
:107DA00082E08083CFE0DFE003C0F801618172816F
:107DB000FE012196E4918E2F0E94D62EFFE0C03363
:107DC000DF0799F781E0DF91CF911F910F9108951F
:107DD0000F931F93CF93DF938C01FC01808182303E
:107DE00031F080E0DF91CF911F910F910895618173
:107DF000728161157105A9F383E08083C6EADEE034
:107E000003C0F80161817281FE012196E4918E2FF9
:107E10000E94D62EFFE0CE30DF0799F781E0DF9198
:107E2000CF911F910F9108950F931F93CF93DF93DD
:107E30008C01FC018081823031F080E0DF91CF91B4
:107E40001F910F9108956181728161157105A9F3E8
:107E500081E08083C7E9DEE003C0F80161817281BF
:107E6000FE012196E4918E2F0E94D62EFEE0C53AA7
:107E7000DF0799F781E0DF91CF911F910F9108956E
:107E80000F931F93CF93DF938C01FC01808181308E
:107E900031F080E0DF91CF911F910F9108956181C2
:107EA000728161157105A9F382E08083CEE4DEE082
:107EB00003C0F80161817281FE012196E4918E2F49
:107EC0000E94D62EFEE0C639DF0799F781E0DF91E8
:107ED000CF911F910F9108950F931F93CF93DF932D
:107EE0008C010097D1F1F8018081882361F0823004
:107EF00081F1833051F1813061F0F8011082F80195
:107F000080818823A1F781E0DF91CF911F910F91AC
:107F10000895F801618172816115710571F3C8E3FB
:107F2000DEE003C0F80161817281FE012196E491D7
:107F30008E2F0E94D62EFEE0CD34DF0799F7F80190
:107F4000818192810E949528D8CFC8010E94BC3EB1
:107F5000CACFC8010E94143FC6CF80E0DF91CF9105
:107F60001F910F9108950F931F93CF93DF938B0170
:107F70006115710539F1DB011C9212961C921E925B
:107F8000119761E60E94A133F80192838183892BC6
:107F9000C9F081E08083C1E4DDE0FE012196E49137
:107FA000D80111966D917C9112978E2F0E94D62E3A
:107FB000BEE0C733DB0789F781E0DF91CF911F91E6
:107FC0000F91089580E0DF91CF911F910F91089557
:107FD000CF93DF93EC018881833071F08130E1F041
:107FE000813080F485E992E0BE010E94B33F813088
:107FF00061F48881833091F7CE010E942E3DDF919C
:10800000CF910895823021F080E0DF91CF910895E3
:10801000CE010E94E83EEBCFCE010E94403FE7CF69
:108020002F923F924F925F926F927F928F929F9288
:10803000AF92BF92CF92DF92EF92FF920F931F9376
:10804000DF93CF93CDB7DEB7C456D0400FB6F894C8
:10805000DEBF0FBECDBF6C01009721F080914D04B3
:108060008823D9F480E0CC59DF4F0FB6F894DEBFF7
:108070000FBECDBFCF91DF911F910F91FF90EF9079
:10808000DF90CF90BF90AF909F908F907F906F9038
:108090005F904F903F902F900895D6018C91833040
:1080A00009F711968D919C911297892BD9F2E09046
:1080B0004504F0904604009147041091480417FDD0
:1080C0001DC23BE2832E912CC801B70120E836E99E
:1080D00048E950E00E946744562E472E382E292E3C
:1080E0003E010894611C711CEDB7FEB73C970FB6BA
:1080F000F894FEBF0FBEEDBFADB6BEB60894A11C8E
:10810000B11C7282618281EA92E0D50113969C9340
:108110008E93129715969C928E921497C801B70170
:1081200020E836E948E950E00E946744C90137FD7C
:10813000E9C1F50197838683652D742D832D922DDA
:1081400020E137E240E050E00E946744C90137FD7A
:10815000E1C1D50119969C938E931897652D742DC6
:10816000832D922D20E137E240E050E00E946744E9
:108170002AE030E040E050E00E946744C90137FD4A
:10818000C5C1F501938782870E94FC448DB79EB7D5
:108190000C960FB6F8949EBF0FBE8DBFD6011196F8
:1081A0006D917C911297C3010E94942FE09041043D
:1081B000F0904204009143041091440417FD9AC1C9
:1081C0009BE2892E912CC801B70120E836E948E9E5
:1081D00050E00E946744562E472E382E292EEDB7C8
:1081E000FEB73C970FB6F894FEBF0FBEEDBFADB61D
:1081F000BEB60894A11CB11C728261828DEB92E024
:10820000D50113969C938E93129715969C928E92FD
:108210001497C801B70120E836E948E950E00E9408
:108220006744C90137FD82C1F50197838683652DB7
:10823000742D832D922D20E137E240E050E00E9422
:108240006744C90137FD6EC1D50119969C938E9381
:108250001897652D742D832D922D20E137E240E093
:1082600050E00E9467442AE030E040E050E00E9485
:108270006744C90137FD52C1F501938782870E9487
:10828000FC448DB79EB70C960FB6F8949EBF0FBEF8
:108290008DBFD60111966D917C911297C3010E94FA
:1082A000942FEDB7FEB770970FB6F894FEBF0FBED0
:1082B000EDBF3196ADB7BEB712967C926E92119714
:1082C00085ED92E09383828380919E0690919F0634
:1082D000958384838091A006868317828091A1066E
:1082E000808711868091A206828713868091A306DB
:1082F000848715868091A406868717860E94FC4491
:10830000EDB7FEB770960FB6F894FEBF0FBEEDBF87
:10831000D60111966D917C911297C3010E94942F02
:1083200000D000D000D0EDB7FEB73196ADB7BEB7E4
:1083300012967C926E92119783E093E093838283EE
:1083400080914F04848315820E94FC44EDB7FEB7F0
:1083500036960FB6F894FEBF0FBEEDBFD60111964C
:108360006D917C911297C3010E94942FD301E3E198
:10837000F3E08FE001900D928150E1F7F601618109
:108380007281C3010E94942F00D000D000D00DB79D
:108390001EB70F5F1F4FADB7BEB712967C926E929D
:1083A000119782E293E0F8019383828360916504E0
:1083B00070916604809167049091680420EA36E821
:1083C00041E050E00E946744D80115963C932E93FB
:1083D00014970E94FC44EDB7FEB736960FB6F8949A
:1083E000FEBF0FBEEDBFD60111966D917C91129725
:1083F000C3010E94942F00D000D000D0EDB7FEB78B
:108400003196ADB7BEB712967C926E9211978AE301
:1084100093E09383828380916104909162049583B9
:1084200084830E94FC44EDB7FEB736960FB6F894ED
:10843000FEBF0FBEEDBFD60111966D917C911297D4
:10844000C3010E94942F2091000130910101EDB7EA
:10845000FEB738970FB6F894FEBF0FBEEDBF31964A
:10846000ADB7BEB712967C926E9211978AE593E0F3
:1084700093838283C9016AE070E00E94324464837E
:108480001582C9016AE070E00E9432448683178237
:108490000E94FC44EDB7FEB738960FB6F894FEBFC5
:1084A0000FBEEDBFD60111966D917C911297C3015D
:1084B0000E94942FD301E7E7F3E080E101900D9251
:1084C0008150E1F7F60161817281C3010E94942F0E
:1084D000D301E7E8F3E08BE001900D928150E1F7E2
:1084E000D60111966D917C911297C3010E94942F31
:1084F00081E0B9CD8DE2882E912C65CE2DE2822EC1
:10850000912CE2CD909581959F4F13CE90958195BA
:108510009F4F37CE909581959F4F1BCE909581951B
:108520009F4FAACE909581959F4F8ECE9095819525
:108530009F4F7ACE0F931F93CF93DF938C01FC0153
:108540008081833031F080E0DF91CF911F910F91D6
:1085500008956181728161157105A9F382E08083BC
:10856000C9E3D0E103C0F80161817281FE01219667
:10857000E4918E2F0E94D62EF0E1C434DF0799F7E4
:1085800081E0DF91CF911F910F9108950F931F9379
:10859000CF93DF938C01FC018081823031F080E049
:1085A000DF91CF911F910F910895618172816115C3
:1085B0007105A9F383E08083CEE2D0E103C0F80126
:1085C00061817281FE012196E4918E2F0E94D62E48
:1085D000F0E1C833DF0799F781E0DF91CF911F9178
:1085E0000F9108950F931F93CF93DF938C01FC019C
:1085F0008081823031F080E0DF91CF911F910F9127
:1086000008956181728161157105A9F381E080830C
:10861000C5E2D0E103C0F80161817281FE012196BB
:10862000E4918E2F0E94D62EF0E1CD32DF0799F72C
:1086300080E0DF91CF911F910F9108950F931F93C9
:10864000CF93DF938C01FC018081813031F080E099
:10865000DF91CF911F910F91089561817281611512
:108660007105A9F382E08083C6E0D0E103C0F80180
:1086700061817281FE012196E4918E2F0E94D62E97
:10868000F0E1C432DF0799F781E0DF91CF911F91CC
:108690000F9108950F931F93CF93DF938C01009751
:1086A000D1F1F8018081882361F0823081F183303B
:1086B00051F1813061F0F8011082F8018081882346
:1086C000A1F781E0DF91CF911F910F910895F801FB
:1086D000618172816115710571F3CDEFDFE003C037
:1086E000F80161817281FE012196E4918E2F0E9432
:1086F000D62EF0E1C530DF0799F7F801818192812C
:108700000E949528D8CFC8010E949A42CACFC801BA
:108710000E94F242C6CF80E0DF91CF911F910F916E
:108720000895CF93DF93EC018881882319F0CE015F
:108730000E944A4318821A82198281E0DF91CF9108
:1087400008950F931F93CF93DF93EC018B01611575
:10875000710539F1CB010E949143CE0161E60E947F
:10876000A133D80112969C938E931197892BC9F04F
:1087700081E08C93C1E3DFE0FE012196E491D80112
:1087800011966D917C9112978E2F0E94D62EBFE08C
:10879000CC3FDB0789F781E0DF91CF911F910F91EB
:1087A000089580E0DF91CF911F910F910895CF93AD
:1087B000DF93EC018881833071F08130E1F081300A
:1087C00080F482E993E0BE010E94A143813061F40C
:1087D0008881833091F7CE010E941040DF91CF91C4
:1087E0000895823021F080E0DF91CF910895CE018D
:1087F0000E94C642EBCFCE010E941E43E7CF629F8C
:10880000D001739FF001829FE00DF11D649FE00D88
:10881000F11D929FF00D839FF00D749FF00D659FE9
:10882000F00D9927729FB00DE11DF91F639FB00DE8
:10883000E11DF91FBD01CF0111240895AA1BBB1B27
:1088400051E107C0AA1FBB1FA617B70710F0A61B50
:10885000B70B881F991F5A95A9F780959095BC0171
:10886000CD01089597FB092E07260AD077FD04D085
:10887000E5DF06D000201AF4709561957F4F0895CA
:10888000F6F7909581959F4F0895A1E21A2EAA1BA5
:10889000BB1BFD010DC0AA1FBB1FEE1FFF1FA217B0
:1088A000B307E407F50720F0A21BB30BE40BF50BAD
:1088B000661F771F881F991F1A9469F76095709536
:1088C000809590959B01AC01BD01CF01089597FB68
:1088D000092E05260ED057FD04D0D7DF0AD0001C84
:1088E00038F450954095309521953F4F4F4F5F4F4D
:1088F0000895F6F790958095709561957F4F8F4F0D
:108900009F4F0895FC0188279927E89421912032F0
:10891000E9F3293010F02E30C8F32B3241F02D321C
:1089200039F4689404C00E94F444820F911D21918F
:1089300020532A30C0F31EF4909581959F4F0895DF
:10894000FB01DC0102C005900D9241505040D8F768
:108950000895FC014150504030F001900616D1F7C7
:108960003197CF010895882799270895FB01DC01ED
:1089700002C001900D9241505040D8F70895FB017C
:10898000DC014150504030F08D910190801919F474
:108990000020B9F7881B990B0895FA01A191B081C5
:1089A000009719F41097E1F0CD01DC01CD010D9095
:1089B000002011F4C00113C0FB012191222319F002
:1089C0002015D9F7F3CFFB012191201519F41E9240
:1089D000119606C02223C1F70D900020A1F7D00107
:1089E000FA01A193B08308957AE0979F902D879F15
:1089F000802D910D11240895AEE0B0E0E2E0F5E4A1
:108A00000C94AB470D891E8986E08C831A830983F9
:108A10008FEF9FE79E838D839E01275E3F4FCE01A0
:108A200001966F89788DA9010E9420452F81388594
:108A3000020F131FF80110822E96E4E00C94C74732
:108A4000ABE0B0E0E6E2F5E40C949D473C012B017D
:108A50005A01FC0117821682838181FD03C06FEFEA
:108A60007FEFC6C19AE0892E1E010894211C311C9B
:108A7000F3012381F20123FD859123FF81912F01D1
:108A8000882309F4B2C1853239F423FD859123FF8F
:108A900081912F01853229F490E0B3010E941347A0
:108AA000E7CF982FFF24EE249924FFE1FF15D0F0A3
:108AB0009B3269F09C3228F4903259F0933291F451
:108AC0000EC09D3249F0903369F441E024C052E079
:108AD000F52A84E0F82A28C098E0F92A25C0E0E1C8
:108AE000FE2A22C0F7FC29C0892F80538A3070F4F7
:108AF000F6FE05C0989C902C1124980E15C0E89C99
:108B0000E02C1124E80EF0E2FF2A0EC09E3229F478
:108B1000F6FC6BC140E4F42A07C09C3619F450E817
:108B2000F52A02C0983649F4F20123FD959123FFFE
:108B300091912F01992309F0B8CF892F8554833063
:108B400018F08052833038F444E050E0A40EB51E93
:108B50005FE359830FC0933631F0933779F0933543
:108B600009F056C020C0F5018081898342E050E0C1
:108B7000A40EB51E610101E010E012C0F501C08035
:108B8000D180F6FC03C06FEF7FEF02C0692D70E06B
:108B900042E050E0A40EB51EC6010E9408478C01B9
:108BA0005FE7F52214C0F501C080D180F6FC03C058
:108BB0006FEF7FEF02C0692D70E042E050E0A40E3D
:108BC000B51EC6010E94FD468C0150E8F52AF3FE51
:108BD00007C01AC080E290E0B3010E941347EA94F4
:108BE0008E2D90E008171907A8F30EC0F601F7FCC8
:108BF0008591F7FE81916F0190E0B3010E941347C8
:108C0000E110EA94015010400115110579F7EAC00E
:108C1000943611F0993669F5F7FE08C0F501208108
:108C200031814281538184E090E00AC0F501808166
:108C300091819C01442737FD4095542F82E090E0BC
:108C4000A80EB91E9FE6F92257FF09C0509540951E
:108C5000309521953F4F4F4F5F4FE0E8FE2ACA0104
:108C6000B901A1012AE030E00E943F47D82ED21876
:108C700040C0953729F41F2D1F7E2AE030E01DC02B
:108C80001F2D197F9F3661F0903720F4983509F039
:108C9000ACC00FC0903739F0983709F0A6C004C0B7
:108CA00028E030E00AC0106114FD146020E130E0DB
:108CB00004C014FD166020E132E017FF08C0F50182
:108CC000608171818281938144E050E008C0F501A8
:108CD00080819181BC0180E090E042E050E0A40EF0
:108CE000B51EA1010E943F47D82ED2188FE7F82E5B
:108CF000F122F6FE0BC05EEFF522D91438F4F4FE33
:108D000007C0F2FC05C08FEEF82202C01D2D01C085
:108D1000192DF4FE0DC0FE01ED0DF11D8081803393
:108D200019F499EEF92208C01F5FF2FE05C003C0D6
:108D30008F2D867809F01F5F0F2DF3FC14C0F0FE15
:108D40000FC01E1510F09D2C0BC09D2C9E0C911A6F
:108D50001E2D06C080E290E0B3010E9413471F5F02
:108D60001E15C0F304C01E1510F4E11A01C0EE2454
:108D700004FF0FC080E390E0B3010E94134702FF9D
:108D80001DC001FD03C088E790E00EC088E590E0BB
:108D90000BC0802F867891F001FF02C08BE201C0EA
:108DA00080E2F7FC8DE290E0B3010E94134706C019
:108DB00080E390E0B3010E9413479A94D914C0F362
:108DC000DA94F101ED0DF11D808190E0B3010E9474
:108DD0001347DD20A9F706C080E290E0B3010E94AE
:108DE0001347EA94EE20C1F743CEF3016681778101
:108DF000CB012B96E2E10C94B947FC010590615040
:108E000070400110D8F7809590958E0F9F1F0895A0
:108E1000FC016150704001900110D8F78095909549
:108E20008E0F9F1F08950F931F93CF93DF938C0195
:108E3000EB018B8181FF1BC082FF0DC02E813F8122
:108E40008C819D812817390764F4E881F9810193A9
:108E5000F983E88306C0E885F985802F0995892B79
:108E600031F48E819F8101969F838E8302C00FEF24
:108E70001FEFC801DF91CF911F910F910895FA0163
:108E8000AA27283051F1203181F1E8946F936E7F49
:108E90006E5F7F4F8F4F9F4FAF4FB1E03ED0B4E03A
:108EA0003CD0670F781F891F9A1FA11D680F791F7B
:108EB0008A1F911DA11D6A0F711D811D911DA11D8C
:108EC00020D009F468943F912AE0269F112430199C
:108ED000305D3193DEF6CF010895462F4770405D37
:108EE0004193B3E00FD0C9F7F6CF462F4F70405DE6
:108EF0004A3318F0495D31FD4052419302D0A9F741
:108F0000EACFB4E0A6959795879577956795BA953A
:108F1000C9F700976105710508959B01AC010A2E00
:108F200006945795479537952795BA95C9F7620FD7
:108F3000731F841F951FA01D08952F923F924F927B
:108F40005F926F927F928F929F92AF92BF92CF92D9
:108F5000DF92EF92FF920F931F93CF93DF93CDB7E2
:108F6000DEB7CA1BDB0B0FB6F894DEBF0FBECDBF5A
:108F700009942A88398848885F846E847D848C842B
:108F80009B84AA84B984C884DF80EE80FD800C8134
:108F90001B81AA81B981CE0FD11D0FB6F894DEBF17
:0C8FA0000FBECDBFED010895F894FFCF87
:108FAC007800FF0164FFFF0348656C6C6F20576FFE
:108FBC00726C640000000000000000000000000063
:108FCC000000000000000000000000000000000095
:108FDC000000000000000000000000000000000085
:108FEC000000000000000000000000000000000075
:108FFC000000000000000000000000001F00000046
:10900C003C0000005B0000007900000098000000AC
:10901C00B6000000D5000000F400000012010000B2
:10902C00310100004F0100006E0100000000000043
:10903C001F0000003B0000005A00000078000000F8
:10904C0097000000B5000000D4000000F300000001
:10905C0011010000300100004E0100006D01000004
:10906C000120202020202020202020202020202013
:10907C0020000073657474696E67732E696E6900E5
:10908C003D002573203D2025640D0A000D0A0000CB
:10909C004B4D4C4C6F6767696E6720202020202059
:1090AC000001F401F401000060EA014750584C6FD4
:1090BC006767696E672020202020200001E803E804
:1090CC0003000060EA4C4F472F25303469253032BD
:1090DC0069253032692F4750582F4750532530356A
:1090EC00692E475058004C4F472F25303469253096
:1090FC003269253032692F4B4D4C2F475053253058
:10910C0035692E4B4D4C00F401E8030D0A256325FF
:10911C00642E252E3364252E33642C0025632564A0
:10912C002E252E3364252E33642C00256325642EC6
:10913C00252E33640064656661756C742E6B6D6CE2
:10914C00003C74726B7074206C61743D2225632535
:10915C00642E252E3364252E33642220006C6F6E12
:10916C003D22256325642E252E3364252E3364225F
:10917C00203E0D0A003C74696D653E253034642D2B
:10918C00253032642D2530326454253032643A2532
:10919C003032643A253032645A3C2F74696D653E26
:1091AC000D0A003C7361743E25643C2F7361743E60
:1091BC000D0A003C657874656E73696F6E733E0DB5
:1091CC000A003C436F757273653E253033643C2F47
:1091DC00436F757273653E0D0A003C47726F756E76
:1091EC006453706565643E25643C2F47726F756EE1
:1091FC006453706565643E0D0A003C566F6C746177
:10920C0067653E25642E253031643C2F566F6C7497
:10921C006167653E0D0A003C2F657874656E736955
:10922C006F6E733E0D0A003C2F74726B70743E0DA2
:0E923C000A0064656661756C742E67707800B8
:00000001FF
